:020000040800F2
:100000000050002025250008DD230008E323000818
:10001000E9230008EF230008F52300080000000092
:10002000000000000000000000000000FB230008AA
:100030000724000800000000132400081F24000803
:100040006D2500086D2500086D2500086D25000848
:100050006D2500086D2500086D2500086D25000838
:100060006D2500086D2500086D2500086D25000828
:100070006D2500086D2500086D2500086D25000818
:100080006D2500086D2500082D2400086D25000849
:100090006D2500086D2500086D2500086D250008F8
:1000A0006D2500086D2500086D2500086D250008E8
:1000B0006D2500086D2500086D2500086D250008D8
:1000C0006D2500086D2500086D2500086D250008C8
:1000D000892400086D2500086D2500086D2500089D
:1000E0009D2400086D2500086D2500080000000013
:1000F0000000000000000000000000000000000000
:0C01000000000000000000005FF808F1A3
:10010C0010B5054C237833B9044B13B10448AFF345
:10011C0000800123237010BDC800002000000000E7
:10012C006C73000808B5034B1BB103490348AFF3CC
:10013C00008008BD00000000CC0000206C7300089B
:10014C00034613F8012B002AFBD1181A013870470B
:10015C0070B54FF0FF0C4CF4E06C1CEA11541DBF51
:10016C001CEA135594EA0C0F95EA0C0F00F0DEF81C
:10017C002C4481EA030621EA4C5123EA4C5350EA01
:10018C00013518BF52EA033541F4801143F4801352
:10019C0038D0A0FB02CE4FF00005E1FB02E506F0E3
:1001AC000042E0FB03E54FF00006E1FB03569CF038
:1001BC00000F18BF4EF0010EA4F1FF04B6F5007F3E
:1001CC0064F5407404D25FEA4E0E6D4146EB0606B0
:1001DC0042EAC62141EA55514FEAC52040EA5E5039
:1001EC004FEACE2EB4F1FD0C88BFBCF5E06F1ED8E3
:1001FC00BEF1004F08BF5FEA500E50F1000041EB1A
:10020C00045170BD06F0004646EA010140EA0200C6
:10021C0081EA0301B4EB5C04C2BFD4EB0C0541EAE8
:10022C00045170BD41F480114FF0000E013C00F3FD
:10023C00AB8014F1360FDEBF002001F0004170BD21
:10024C00C4F10004203C35DA0C341BDC04F114043A
:10025C00C4F1200500FA05F320FA04F001FA05F2C6
:10026C0040EA020001F0004221F0004110EBD37093
:10027C0021FA04F642EB06015EEA430E08BF20EABF
:10028C00D37070BDC4F10C04C4F1200500FA04F362
:10029C0020FA05F001FA04F240EA020001F00041F4
:1002AC0010EBD37041F100015EEA430E08BF20EA67
:1002BC00D37070BDC4F1200500FA05F24EEA020EAF
:1002CC0020FA04F301FA05F243EA020321FA04F0DE
:1002DC0001F0004121FA04F220EA020000EBD37095
:1002EC005EEA430E08BF20EAD37070BD94F0000F95
:1002FC000FD101F00046400041EB010111F4801FC9
:10030C0008BF013CF7D041EA060195F0000F18BF79
:10031C00704703F00046520043EB030313F4801FB5
:10032C0008BF013DF7D043EA0603704794EA0C0F6F
:10033C000CEA135518BF95EA0C0F0CD050EA410685
:10034C0018BF52EA4306D1D181EA030101F0004102
:10035C004FF0000070BD50EA410606BF104619462A
:10036C0052EA430619D094EA0C0F02D150EA013636
:10037C0013D195EA0C0F05D152EA03361CBF104677
:10038C0019460AD181EA030101F0004141F0FE4116
:10039C0041F470014FF0000070BD41F0FE4141F49A
:1003AC00780170BD81F0004102E000BF83F0004392
:1003BC0030B54FEA41044FEA430594EA050F08BFF4
:1003CC0090EA020F1FBF54EA000C55EA020C7FEAB8
:1003DC00645C7FEA655C00F0E2804FEA5454D4EB35
:1003EC005555B8BF6D420CDD2C4480EA020281EAFF
:1003FC00030382EA000083EA010180EA020281EA37
:10040C000303362D88BF30BD11F0004F4FEA013188
:10041C004FF4801C4CEA113102D0404261EB410197
:10042C0013F0004F4FEA03334CEA133302D052421D
:10043C0063EB430394EA050F00F0A780A4F10104D9
:10044C00D5F1200E0DDB02FA0EFC22FA05F2801813
:10045C0041F1000103FA0EF2801843FA05F35941F9
:10046C000EE0A5F120050EF1200E012A03FA0EFC78
:10047C0028BF4CF0020C43FA05F3C01851EBE371A2
:10048C0001F0004507D54FF0000EDCF1000C7EEBBF
:10049C0000006EEB0101B1F5801F1BD3B1F5001FFD
:1004AC000CD349085FEA30004FEA3C0C04F101041C
:1004BC004FEA445212F5800F80F09A80BCF1004F45
:1004CC0008BF5FEA500C50F1000041EB045141EAC7
:1004DC00050130BD5FEA4C0C404141EB0101013C90
:1004EC0028BFB1F5801FE9D291F0000F04BF01467F
:1004FC000020B1FA81F308BF2033A3F10B03B3F151
:10050C0020020CDA0C3208DD02F1140CC2F10C02E0
:10051C0001FA0CF021FA02F10CE002F11402D8BF3E
:10052C00C2F1200C01FA02F120FA0CFCDCBF41EA0A
:10053C000C019040E41AA2BF01EB0451294330BDD9
:10054C006FEA04041F3C1CDA0C340EDC04F11404B6
:10055C00C4F1200220FA04F001FA02F340EA03008D
:10056C0021FA04F345EA030130BDC4F10C04C4F1D3
:10057C00200220FA02F001FA04F340EA03002946B3
:10058C0030BD21FA04F0294630BD94F0000F83F4FD
:10059C00801306BF81F480110134013D4EE77FEAE0
:1005AC00645C18BF7FEA655C29D094EA050F08BF2C
:1005BC0090EA020F05D054EA000C04BF194610460D
:1005CC0030BD91EA030F1EBF0021002030BD5FEA51
:1005DC00545C05D14000494128BF41F0004130BD79
:1005EC0014F580043CBF01F5801130BD01F00045CD
:1005FC0045F0FE4141F470014FF0000030BD7FEA40
:10060C00645C1ABF194610467FEA655C1CBF0B463A
:10061C00024650EA013406BF52EA033591EA030F51
:10062C0041F4002130BD00BF90F0000F04BF002149
:10063C00704730B54FF4806404F132044FF000057C
:10064C004FF0000150E700BF90F0000F04BF0021F5
:10065C00704730B54FF4806404F1320410F000455B
:10066C0048BF40424FF000013EE700BF42004FEA56
:10067C00E2014FEA31014FEA02701FBF12F07F43D3
:10068C0093F07F4F81F06051704732F07F4208BF8A
:10069C00704793F07F4F04BF41F40021704730B591
:1006AC004FF4607401F0004521F000411CE700BFDD
:1006BC0050EA010208BF704730B54FF000050AE060
:1006CC0050EA010208BF704730B511F0004502D561
:1006DC00404261EB41014FF4806404F132045FEA63
:1006EC00915C3FF4D8AE4FF003025FEADC0C18BF0C
:1006FC0003325FEADC0C18BF033202EBDC02C2F1FE
:10070C00200300FA03FC20FA02F001FA03FE40EA8F
:10071C000E0021FA02F11444BDE600BF4A0011D2CA
:10072C0012F5001211D20DD56FF47873B3EB62523F
:10073C000ED44FEAC12343F0004343EA505323FA4B
:10074C0002F070474FF00000704750EA013002D1C0
:10075C004FF0FF3070474FF00000704780F00040C2
:10076C0002E000BF81F0004142001FBF5FEA41037D
:10077C0092EA030F7FEA226C7FEA236C6AD04FEA7D
:10078C001262D2EB1363C1BFD218414048404140C2
:10079C00B8BF5B42192B88BF704710F0004F40F474
:1007AC00000020F07F4018BF404211F0004F41F490
:1007BC00000121F07F4118BF494292EA030F3FD05C
:1007CC00A2F1010241FA03FC10EB0C00C3F120036F
:1007DC0001FA03F100F0004302D5494260EB4000FE
:1007EC00B0F5000F13D3B0F1807F06D340084FEA69
:1007FC00310102F10102FE2A51D2B1F1004F40EB5E
:10080C00C25008BF20F0010040EA030070474900C5
:10081C0040EB0000013A28BFB0F5000FEDD2B0FA62
:10082C0080FCACF1080CB2EB0C0200FA0CF0AABF85
:10083C0000EBC25052421843BCBFD0401843704723
:10084C0092F0000F81F4000106BF80F40000013229
:10085C00013BB5E74FEA41037FEA226C18BF7FEA00
:10086C00236C21D092EA030F04D092F0000F08BF42
:10087C000846704790EA010F1CBF0020704712F029
:10088C007F4F04D1400028BF40F00040704712F168
:10089C0000723CBF00F50000704700F0004343F0CD
:1008AC00FE4040F4000070477FEA226216BF084603
:1008BC007FEA23630146420206BF5FEA412390EAC6
:1008CC00010F40F4800070474FF0000304E000BFBC
:1008DC0010F0004348BF40425FEA000C08BF70476D
:1008EC0043F0964301464FF000001CE050EA010231
:1008FC0008BF70474FF000030AE000BF50EA010246
:10090C0008BF704711F0004302D5404261EB410132
:10091C005FEA010C02BF84460146002043F0B64357
:10092C0008BFA3F18053A3F50003BCFA8CF2083A7C
:10093C00A3EBC25310DB01FA02FC634400FA02FC85
:10094C00C2F12002BCF1004F20FA02F243EB02008C
:10095C0008BF20F00100704702F1200201FA02FCEE
:10096C00C2F1200250EA4C0021FA02F243EB0200E1
:10097C0008BF20EADC7070474FF0FF0C1CEAD05225
:10098C001EBF1CEAD15392EA0C0F93EA0C0F6FD0E6
:10099C001A4480EA010C400218BF5FEA41211ED0C4
:1009AC004FF0006343EA501043EA5111A0FB0131B0
:1009BC000CF00040B1F5000F3EBF490041EAD37185
:1009CC005B0040EA010062F17F02FD2A1DD8B3F101
:1009DC00004F40EBC25008BF20F00100704790F070
:1009EC00000F0CF0004C08BF49024CEA502040EAC2
:1009FC0051207F3AC2BFD2F1FF0340EAC250704788
:100A0C0040F400004FF00003013A5DDC12F1190FC5
:100A1C00DCBF00F000407047C2F10002410021FA37
:100A2C0002F1C2F1200200FA02FC5FEA310040F14F
:100A3C00000053EA4C0308BF20EADC70704792F0C8
:100A4C00000F00F0004C02BF400010F4000F013A00
:100A5C00F9D040EA0C0093F0000F01F0004C02BFFB
:100A6C00490011F4000F013BF9D041EA0C018FE76A
:100A7C000CEAD15392EA0C0F18BF93EA0C0F0AD070
:100A8C0030F0004C18BF31F0004CD8D180EA010096
:100A9C0000F00040704790F0000F17BF90F0004F2F
:100AAC00084691F0000F91F0004F14D092EA0C0F11
:100ABC0001D142020FD193EA0C0F03D14B0218BFA4
:100ACC00084608D180EA010000F0004040F0FE40EA
:100ADC0040F40000704740F0FE4040F44000704786
:100AEC004FF0FF0C1CEAD0521EBF1CEAD15392EA05
:100AFC000C0F93EA0C0F69D0A2EB030280EA010CF5
:100B0C0049024FEA402037D04FF0805343EA11118D
:100B1C0043EA10130CF000408B4238BF5B0042F1EB
:100B2C007D024FF4000C8B4224BF5B1A40EA0C0090
:100B3C00B3EB510F24BFA3EB510340EA5C00B3EBC2
:100B4C00910F24BFA3EB910340EA9C00B3EBD10FB0
:100B5C0024BFA3EBD10340EADC001B0118BF5FEA02
:100B6C001C1CE0D1FD2A3FF650AF8B4240EBC2502B
:100B7C0008BF20F0010070470CF0004C4CEA5020EC
:100B8C007F32C2BFD2F1FF0340EAC250704740F43B
:100B9C0000004FF00003013A37E792F0000F00F02D
:100BAC00004C02BF400010F4000F013AF9D040EAAB
:100BBC000C0093F0000F01F0004C02BF490011F43F
:100BCC00000F013BF9D041EA0C0195E70CEAD15337
:100BDC0092EA0C0F08D142027FF47DAF93EA0C0F1E
:100BEC007FF470AF084676E793EA0C0F04D14B0202
:100BFC003FF44CAF08466EE730F0004C18BF31F0B4
:100C0C00004CCAD130F000427FF45CAF31F00043AD
:100C1C007FF43CAF5FE700BF4FF0FF3C06E000BF46
:100C2C004FF0010C02E000BF4FF0010C4DF804CD69
:100C3C004FEA40024FEA41037FEA226C18BF7FEA79
:100C4C00236C11D001B052EA530C18BF90EA010F7B
:100C5C0058BFB2EB030088BFC81738BF6FEAE1700A
:100C6C0018BF40F0010070477FEA226C02D15FEAA6
:100C7C00402C05D17FEA236CE4D15FEA412CE1D012
:100C8C005DF8040B704700BF844608466146FFE7D9
:100C9C000FB5FFF7C9FF002848BF10F1000F0FBDBB
:100CAC004DF808EDFFF7F4FF0CBF012000205DF8B4
:100CBC0008FB00BF4DF808EDFFF7EAFF34BF012039
:100CCC0000205DF808FB00BF4DF808EDFFF7E0FFD2
:100CDC0094BF012000205DF808FB00BF4DF808ED23
:100CEC00FFF7D2FF94BF012000205DF808FB00BF86
:100CFC004DF808EDFFF7C8FF34BF012000205DF868
:100D0C0008FB00BF80B582B000AF0346FB804FF4F8
:100D1C008051154802F0C6FC0346002B1FD1134B23
:100D2C001B78002B0BD0124B1B78002B07D0114BD0
:100D3C001B68114A13600D4B00221A7006E00C4B15
:100D4C001B78002B02D00C4B0C4A1A600A4B19680A
:100D5C000B4B1A684FF484730A4803F007FF00BF6B
:100D6C000837BD4680BD00BF000C0140E5000020E7
:100D7C00E6000020100500200805002014050020C6
:100D8C000C050020A406002080B485B000AF78606C
:100D9C000B46FB700023FB6007E0FB687A6813448A
:100DAC00FA781A70FB680133FB60FB68B3F5847F3B
:100DBC00F3DB00BF00BF1437BD4680BC704700009A
:100DCC0080B500AF074B00221A70064B1B781846F3
:100DDC0000F044F8AA210448FFF7D6FF00F006F80B
:100DEC0000BF80BDE6000020F802002080B582B074
:100DFC0000AF194BFA221A70174BAF225A70164BD0
:100E0C0003229A70144BFF2283F80221124B0D22FD
:100E1C0083F803214FF482710F4800F0C3FF786010
:100E2C007B681B0EDAB20C4B83F804217B681B0C1D
:100E3C00DAB2094B83F805217B681B0ADAB2064B40
:100E4C0083F806217B68DAB2034B83F8072100BFD5
:100E5C000837BD4680BD00BF1405002080B483B0A8
:100E6C0000AF0346FB71FB79002B03D0074B084AFC
:100E7C001A6005E0074B084A1A60044B074A1A60CF
:100E8C0000BF0C37BD4680BC704700BF0C0500206E
:100E9C000004002008050020F8020020E8000020D3
:100EAC0080B582B000AF78607B681B68114A9342B2
:100EBC001BD1114B1B78002B03D00F4B00221A7047
:100ECC000EE00D4B01221A700C4A0D4B10461946C0
:100EDC004FF484731A4605F0C1FD0A4B01221A70B7
:100EEC00054B1B781846FFF7B9FF00BF0837BD4606
:100EFC0080BD00BF00380040E6000020F00100205B
:100F0C00E8000020E400002090B587B000AF01F0AD
:100F1C0029FB00F045F900F03BFB00F011FA00F062
:100F2C000DFB00F099F900F0D5F900F0B9FA00F0DA
:100F3C0039FA01221821884802F0CBFB00F05EFF41
:100F4C00864B1B6847F248125A62844804F02CFA0C
:100F5C00834801F06BFD6421814801F061FC814BF9
:100F6C001B78002B04D07F4B00221A7000F058FD28
:100F7C007D4B1B78302B0CD101220421764802F0DA
:100F8C00A8FB05F053FA794B00221A70784B00221B
:100F9C001A80754B1B78312B07D1012204216E4826
:100FAC0002F097FB734B01221A706F4B1B78322B9C
:100FBC0007D101220421684802F08BFB6D4B002203
:100FCC001A70694B1B78332B14D10122042162480F
:100FDC0002F07FFB644B5B781946674B1B88002241
:100FEC00664805F095FC644B1A8864236349644891
:100FFC0004F0FDFF5C4B00221A70002204215648BD
:10100C0002F067FB5B4B1B78002BA8D05D4B1B7869
:10101C00DBB2012BA3D15B4B00221A705A4B1B88FD
:10102C007B827B8A1846FFF74FFC04467B8AC3F50C
:10103C007F630F331846FFF74BFC034619462046D7
:10104C00FFF74EFD0346FB6009237B6147E04F4AE7
:10105C007B6952F823301946F868FFF735FE0346D2
:10106C00002B39D07B690133484A52F82320474979
:10107C007B6951F8233019461046FFF773FB034682
:10108C0019464348FFF72CFD0346BB607B695A1E8B
:10109C0013469B0013441846FFF71AFC04463B4AC0
:1010AC007B6952F82330B9681846FFF765FC034694
:1010BC0019462046FFF756FB03467B60F968B86873
:1010CC00FFF75AFC034679681846FFF74DFB0346B9
:1010DC001A46304B1A6005E07B69013B7B617B69EA
:1010EC00002BB4DA2B4B1B681846FFF7BFFA4FF0F6
:1010FC000002294BFFF72CF802460B461046194606
:10110C00FFF70CFB03469AB2244B1A80184B1B8832
:10111C009BB21946154B1B785B001A4602231F48DD
:10112C0005F0A8F9114B1B780133DAB20F4B1A708A
:10113C000E4B1B787F2B09D10D4B1B889BB20133B7
:10114C009AB20B4B1A80094B00221A7004210248E8
:10115C0002F0D7FA03E700BF000801404407002063
:10116C001C060020E4000020D8080020D508002030
:10117C00D2080020D00800200C0A0020D007002044
:10118C008C070020D4080020000A0020000000205A
:10119C000000A040E408002000005940E8080020AE
:1011AC0080B594B000AF07F128032822002118461F
:1011BC0005F062FC07F1140300221A605A609A6071
:1011CC00DA601A613B1D00221A605A609A60DA607C
:1011DC000123BB624FF48033FB6200233B6301238A
:1011EC00BB6302237B644FF48033BB644FF4E01386
:1011FC00FB6407F12803184602F0B4FA0346002BEF
:10120C0001D000F027FA0F237B610223BB6100237E
:10121C00FB614FF480633B6200237B6207F1140394
:10122C000221184602F020FD0346002B01D000F0ED
:10123C0011FA02237B604FF40043FB603B1D184600
:10124C0002F0AAFE0346002B01D000F003FA00BF07
:10125C005037BD4680BD000080B584B000AF3B1D4B
:10126C0000221A605A609A60184B194A1A60174B80
:10127C0000229A60154B00221A73144B00221A7527
:10128C00124B4FF40022DA61104B00225A600F4BC4
:10129C0001221A610D4801F0EBF90346002B01D035
:1012AC0000F0D8F901237B600123BB600023FB60B5
:1012BC003B1D1946054801F051FD0346002B01D09A
:1012CC0000F0C8F900BF1037BD4680BD1C060020D9
:1012DC000024014080B500AF174B184A1A60164B1A
:1012EC004FF482725A60144B00229A60124B002207
:1012FC00DA60114B00221A610F4B00225A610E4B1F
:10130C004FF400729A610C4B2022DA610A4B0022D6
:10131C001A62094B00225A62074B00229A62064B52
:10132C000A22DA62044802F0ADFF0346002B01D01A
:10133C0000F090F900BF80BD4C0600200030014049
:10134C0080B500AF154B164A1A60144B00225A6038
:10135C00124B00229A60114B0022DA600F4B0022D4
:10136C001A610E4B00225A610C4B4FF400729A61B9
:10137C000A4B00221A62094B00225A62074B0022C8
:10138C009A62064B0A22DA62044802F07BFF03469B
:10139C00002B01D000F05EF900BF80BDA406002038
:1013AC000038004080B58EB000AF07F12803002252
:1013BC001A605A609A60DA6007F1200300221A6002
:1013CC005A603B1D00221A605A609A60DA601A61FA
:1013DC005A619A61314B4FF080421A602F4B482270
:1013EC005A602E4B00229A602C4B40F2F512DA60B8
:1013FC002A4B00221A61294B00229A61274803F0DC
:10140C0083FF0346002B01D000F024F94FF48053E6
:10141C00BB6207F128031946204804F0D5F90346AE
:10142C00002B01D000F016F91C4804F007F8034615
:10143C00002B01D000F00EF90821184804F056F8E2
:10144C000346002B01D000F005F900233B6200237A
:10145C007B6207F120031946104804F01DFD03467A
:10146C00002B01D000F0F6F860237B600123BB60F9
:10147C000223FB6000237B613B1D002219460748B9
:10148C0004F0E4F80346002B01D000F0E3F8034825
:10149C0000F022FF00BF3837BD4680BDFC0600209F
:1014AC0080B586B000AF07F1080300221A605A60BD
:1014BC009A60DA603B4600221A605A601D4B1E4A45
:1014CC001A601C4B4FF6FF725A601A4B00229A603E
:1014DC00184B47F23052DA60164B00221A61154B4A
:1014EC0000229A61134803F00FFF0346002B01D032
:1014FC0000F0B0F84FF48053BB6007F108031946B5
:10150C000C4804F061F90346002B01D000F0A2F85E
:10151C0030233B6000237B603B461946054804F0B2
:10152C00BBFC0346002B01D000F094F800BF183729
:10153C00BD4680BD440700200004004080B500AFCC
:10154C00114B124A1A60104B4FF47A325A600E4B00
:10155C0000229A600C4B0022DA600B4B00221A61BD
:10156C00094B0C225A61084B00229A61064B00224F
:10157C00DA61054804F0EEFC0346002B01D000F0C4
:10158C0069F800BF80BD00BF8C0700200038014007
:10159C0080B588B000AF07F1100300221A605A60C2
:1015AC009A60DA60274B9B69264A43F020039361CB
:1015BC00244B9B6903F02003FB60FB68214B9B6968
:1015CC00204A43F0040393611E4B9B6903F0040310
:1015DC00BB60BB681B4B9B691A4A43F008039361C1
:1015EC00184B9B6903F008037B607B6800221C216D
:1015FC00154802F06EF81C233B6101237B6100232C
:10160C00BB610223FB6107F1100319460E4801F080
:10161C00C5FE4FF480533B610C4B7B610023BB61D7
:10162C0007F1100319460A4801F0B8FE0022012107
:10163C00282001F006FE282001F01FFE00BF2037F5
:10164C00BD4680BD00100240000801400000211082
:10165C00000C014080B400AF72B600BFFEE7000082
:10166C0080B483B000AF234B1B78BB71224B1B881B
:10167C009BB27B71214B1A687B799A420AD11F4B22
:10168C0093F904301A46BB799A4203D11B4B0022C2
:10169C005A712BE0194B1A687B799A4206D1BB79A7
:1016AC00002B03D1154B00225A711FE0134B1A6803
:1016BC007B799A4201D07F23BB71104B93F9043094
:1016CC00B3F1FF3F02D10023FB7106E00B4B93F902
:1016DC0004300133DBB25B00FB71BB795B00DAB227
:1016EC00FB79D31ADAB2054B5A7100BF0C37BD46E1
:1016FC0080BC7047D5080020D208002028000020AC
:10170C0080B483B000AF0346FB71044AFB791370BD
:10171C0000BF0C37BD4680BC704700BFF4090020E9
:10172C0080B582B000AF4FF4847200211F4805F0E1
:10173C00A3F91E4BFA221A701C4BAA225A7000F005
:10174C003DF8FFF78DFF1A4B5A79184B9A70174BCF
:10175C00FF2283F80221154B0B2283F803214FF44F
:10176C008271124800F01EFB78607B681B0EDAB2A7
:10177C000E4B83F804217B681B0CDAB20B4B83F8FD
:10178C0005217B681B0ADAB2084B83F806217B68BB
:10179C00DAB2064B83F80721064B044A1A60064B53
:1017AC0001221A7000BF0837BD4680BDEC0800202E
:1017BC002800002010050020E500002080B582B034
:1017CC0000AF3B4B5B79002B6ED0012204213948D2
:1017DC0001F07FFF364B1968374B1B8800223748C6
:1017EC0005F096F8324B93F90430B3F1FF3F02D178
:1017FC000023FB7106E02E4B93F904300133DBB26E
:10180C005B00FB712A4B5A79FB791344DBB2013B29
:10181C007B700323BB80FB797B800BE07A88BB88D1
:10182C002649895C264AD1547B8801337B80BB884E
:10183C000133BB807B789BB27A889A42EED91C4BE1
:10184C0093F90430B3F1FF3F09D1194B5B795B0875
:10185C00DBB2013BDBB25AB2154B1A710CE0144BE4
:10186C0093F90430DAB2124B5B795B08DBB21344A8
:10187C00DBB25AB20E4B1A710D4B93F904307E2B1E
:10188C0013D10B4B1B684FF6FF72934203D1084BDD
:10189C0000221A6004E0064B1B680133044A1360F3
:1018AC00034BFF221A7100E000BF0837BD4680BD14
:1018BC0028000020000801400C0A0020D00700205E
:1018CC00EC08002080B584B000AF03460A46FB80CC
:1018DC001346BB804FF484720021214805F0CCF8EC
:1018EC001F4BFA221A701E4BAF225A70FB88DAB2C9
:1018FC001B4B9A70BB88A22B03D11A4B5A79184BED
:10190C00DA70174BFF2283F80221154B0D2283F856
:10191C0003214FF48271124800F044FAF860FB681E
:10192C001B0EDAB20E4B83F80421FB681B0CDAB2E7
:10193C000B4B83F80521FB681B0ADAB2084B83F8C2
:10194C000621FB68DAB2064B83F80721064B044AE2
:10195C001A60064B01221A7000BF1037BD4680BDBD
:10196C00EC0800202800002010050020E5000020D5
:10197C0080B500AF054800F00FF8054B034A1A601C
:10198C00044B01221A7000BF80BD00BFEC08002080
:10199C0010050020E500002080B584B000AF786011
:1019AC007B6801331B78AA2B07D1FFF759FE7B68A4
:1019BC0002331A4A52791A700BE07B6802331B7897
:1019CC00A22B06D1FFF74CFE7B680333134A5279E6
:1019DC001A704FF48271786800F0E4F9F860FB68D3
:1019EC001A0E7B6803F58273D2B21A70FB681A0C5C
:1019FC007B6803F20513D2B21A70FB681A0A7B6873
:101A0C0003F58373D2B21A707B6803F20713FA687A
:101A1C00D2B21A7000BF1037BD4680BD280000201E
:101A2C0080B500AF00F012FA4FF48271BA4800F0A2
:101A3C0089F9034683F00103DBB2002B04D00021AB
:101A4C00FF20FFF73FFF7CE1B44B1B78052B00F226
:101A5C00788101A252F823F07D1A0008DB1A0008E5
:101A6C00571B0008E51B0008651C0008ED1C00084E
:101A7C00A94B9B78FF2B26D0FF2B00F35981A22B6F
:101A8C0002D0A32B1CD053E100F07CFA0346002BB0
:101A9C0011D0FFF7E5FDA24B5B79002B03D003209F
:101AAC00FFF72EFE02E00120FFF72AFEA2212C20D8
:101ABC00FFF708FF0AE0A2210820FFF703FF05E06B
:101ACC0000F09EFA02E0FFF753FF00BF30E1924BAB
:101ADC009B78FF2B35D0FF2B00F32C81A42B26D029
:101AEC00A42B00F32781A22B02D0A32B1CD021E125
:101AFC0000F048FA0346002B11D0FFF7B1FD884BDC
:101B0C005B79002B03D00320FFF7FAFD02E00120E4
:101B1C00FFF7F6FDA2212C20FFF7D4FE14E0A22142
:101B2C000820FFF7CFFE0FE000F06AFA0CE0A421CA
:101B3C000620FFF7C7FE00F083FA0220FFF7E0FD56
:101B4C0002E0FFF715FF00BFF4E0734B9B78A72B67
:101B5C0018DCA12BC0F2F080A13B062B00F2EC802C
:101B6C0001A252F823F000BF971B0008A31B00082A
:101B7C00C31B0008451D0008451D0008451D000835
:101B8C00C91B0008FF2B23D0D6E00420FFF7B8FDBB
:101B9C00FFF7C6FD1FE0FFF763FD614B5B79002B80
:101BAC0004D0A2210120FFF78DFE14E0A221022017
:101BBC00FFF788FE0FE000F023FA0CE000F04CFA7F
:101BCC00A7210720FFF77EFE0120FFF799FD02E019
:101BDC00FFF7CEFE00BFAFE04F4B9B78A42B11DC80
:101BEC00A12BC0F2AB80A13B032B00F2A78001A27A
:101BFC0052F823F0171C00081D1C0008431C000899
:101C0C00491C0008FF2B23D098E0FFF789FD22E048
:101C1C00FFF726FD424B5B79002B04D0A22101205B
:101C2C00FFF750FE17E0A2210220FFF74BFE012028
:101C3C00FFF766FD0FE000F0E3F90CE0A4210620AD
:101C4C00FFF740FE00F0FCF90420FFF759FD02E01D
:101C5C00FFF78EFE00BF71E02F4B9B78A72B15DC96
:101C6C00A12B6DDBA13B062B6AD801A252F823F005
:101C7C009F1C0008A51C0008CB1C00084D1D00086B
:101C8C004D1D00084D1D0008D11C0008FF2B23D052
:101C9C0056E0FFF745FD22E0FFF7E2FC204B5B79B5
:101CAC00002B04D0A2210120FFF70CFE17E0A2218B
:101CBC000220FFF707FE0220FFF722FD0FE000F0E5
:101CCC009FF90CE000F0C8F9A7210720FFF7FAFDF7
:101CDC000320FFF715FD02E0FFF74AFE00BF2FE0DF
:101CEC000D4B9B78A22B2CD10E4B1B78002B0FD0BD
:101CFC00002204210C4801F0ECFCA3210520FFF785
:101D0C00E1FD0020FFF7FCFC064B00221A7018E0E6
:101D1C00064B00221A7014E0F0010020F409002098
:101D2C0028000020F509002000080140E5000020F3
:101D3C0000BF06E000BF04E000BF02E000BF00E00F
:101D4C0000BF80BD80B584B000AF78600B467B804F
:101D5C007B6803F207131B781A467B6803F58373C1
:101D6C001B781B021A437B6803F205131B781B04B8
:101D7C001A437B6803F582731B781B061343FB60C5
:101D8C004FF48271786800F00DF8B860FA68BB689F
:101D9C009A4201D0002300E0012318461037BD46BB
:101DAC0080BD000080B485B000AF78600B467B80AE
:101DBC004FF0FF33FB600023BB6011E0BB687A6817
:101DCC0013441B781A46FB685340DBB20A4A52F89C
:101DDC002320FB681B0A5340FB60BB680133BB60CC
:101DEC007B88BA689A42E9DBFB68DB4318461437F8
:101DFC00BD4680BC704700BFE076000880B500AFE0
:101E0C00002004F0DFFBFEF7DBFF0021064803F0A7
:101E1C00C7FB012000F008FC00F008F80020FFF7D9
:101E2C006FFC00BF80BD00BFFC06002080B400AF7B
:101E3C00054B1B681A68044B1B6842F001021A60C0
:101E4C0000BFBD4680BC7047FC06002080B400AFCC
:101E5C00054B1B681A68044B1B6842F001021A60A0
:101E6C0000BFBD4680BC7047FC06002080B500AFAB
:101E7C000520FFF745FC074B00221A60054BFF229B
:101E8C001A71044B00225A71034B00221A7000BFC6
:101E9C0080BD00BF28000020E500002090B587B071
:101EAC0000AF354B1B889BB21846FEF70DFD044660
:101EBC00314B1B889BB2C3F57F630F331846FEF77B
:101ECC0007FD034619462046FEF70AFE0346FB6053
:101EDC004FF000037B6109233B6145E0274A3B69D6
:101EEC0052F823301946F868FEF7EEFE0346002B35
:101EFC0037D03B690133214A52F823201F493B69F3
:101F0C0051F8233019461046FEF72CFC03461946AF
:101F1C001B48FEF7E5FD0346BB603B695A1E1346A2
:101F2C009B0013441846FEF7D3FC0446134A3B6946
:101F3C0052F82330B9681846FEF71EFD03461946C1
:101F4C002046FEF70FFC03467B60F968B868FEF785
:101F5C0013FD034619467868FEF706FC03467B61C1
:101F6C0005E03B69013B3B613B69002BB6DA7B69C1
:101F7C0018461C37BD4690BDF609002030000020E5
:101F8C000000A04080B500AF184B01221A70184B0E
:101F9C001B889BB240F6FF72934204D1134B002274
:101FAC001A7000231FE0FFF779FF0346114A1360F4
:101FBC00104B1B6810491846FEF77CFE0346002B9D
:101FCC0008D10C4B1B680D491846FEF791FE0346D1
:101FDC00002B04D0054B00221A70002303E0034BA6
:101FEC0000221A700123184680BD00BFF80900209A
:101FFC00F6090020FC0900200000F04100004842D6
:10200C0080B500AF00F028F8FFF730FF084B002236
:10201C001A70084B00221A8001220421064801F094
:10202C0058FB04F003FA054B01221A7000BF80BD67
:10203C00D5080020D208002000080140F509002036
:10204C0080B400AF034B31221A7000BFBD4680BC78
:10205C00704700BFD808002080B400AF034B322279
:10206C001A7000BFBD4680BC704700BFD808002066
:10207C0080B485B000AF154B9B69144A43F0010343
:10208C009361124B9B6903F00103BB60BB680F4B60
:10209C00DB690E4A43F08053D3610C4BDB6903F0D0
:1020AC0080537B607B680A4B5B68FB60FB6823F0AA
:1020BC00E063FB60FB6843F00073FB60044AFB6861
:1020CC00536000BF1437BD4680BC704700100240FF
:1020DC000000014080B588B000AF786007F11003B4
:1020EC0000221A605A609A60DA607B681B68184A92
:1020FC00934229D1174B9B69164A43F400739361A1
:10210C00144B9B6903F40073FB60FB68114B9B69D8
:10211C00104A43F0040393610E4B9B6903F00403D4
:10212C00BB60BB6802233B6103237B6107F1100397
:10213C001946094801F032F900220121122001F060
:10214C0080F8122001F099F800BF2037BD4680BD01
:10215C0000240140001002400008014080B58AB004
:10216C0000AF786007F1180300221A605A609A6079
:10217C00DA607B681B683B4A934230D13A4B9B69CF
:10218C00394A43F480539361374B9B6903F4805372
:10219C007B617B69344B9B69334A43F00403936145
:1021AC00314B9B6903F004033B613B69A023BB618A
:1021BC000223FB6103237B6207F1180319462B48AA
:1021CC0001F0ECF84023BB610023FB6100233B6270
:1021DC0007F118031946254801F0E0F83EE07B684A
:1021EC001B68234A934239D11F4BDB691E4A43F4C7
:1021FC008043D3611C4BDB6903F48043FB60FB68B9
:10220C00194B9B69184A43F008039361164B9B6961
:10221C0003F00803BB60BB684FF42043BB61002391
:10222C00FB6100233B6207F118031946114801F0CA
:10223C00B5F84FF48043BB610223FB6103237B623F
:10224C0007F1180319460B4801F0A8F800220121E8
:10225C00242000F0F6FF242001F00FF800BF2837EF
:10226C00BD4680BD00300140001002400008014016
:10227C0000380040000C014080B485B000AF78609D
:10228C007B681B68B3F1804F0CD1114BDB69104A92
:10229C0043F00103D3610E4BDB6903F00103FB60D8
:1022AC00FB6810E07B681B680A4A93420BD1084B11
:1022BC00DB69074A43F00203D361054BDB6903F08A
:1022CC000203BB60BB6800BF1437BD4680BC7047BF
:1022DC00001002400004004080B588B000AF786068
:1022EC0007F1100300221A605A609A60DA607B686A
:1022FC001B68B3F1804F17D10D4B9B690C4A43F00F
:10230C00040393610A4B9B6903F00403FB60FB68B5
:10231C0001233B6102237B610223FB6107F1100364
:10232C001946044801F03AF800BF2037BD4680BD7D
:10233C00001002400008014080B588B000AF786002
:10234C0007F1100300221A605A609A60DA607B6809
:10235C001B681C4A934231D11B4B9B691A4A43F4AC
:10236C0080439361184B9B6903F48043FB60FB68CB
:10237C00154B9B69144A43F004039361124B9B6900
:10238C0003F00403BB60BB684FF400733B61022392
:10239C007B610323FB6107F1100319460B4800F026
:1023AC00FDFF4FF480633B6100237B610023BB6125
:1023BC0007F110031946054800F0F0FF00BF203765
:1023CC00BD4680BD003801400010024000080140AD
:1023DC0080B400AFFEE780B400AFFEE780B400AF7E
:1023EC00FEE780B400AFFEE780B400AFFEE780B438
:1023FC0000AF00BFBD4680BC704780B400AF00BFCB
:10240C00BD4680BC704780B400AF00BFBD4680BCE9
:10241C00704780B500AF00F0EBF800BF80BD000046
:10242C0080B500AF0F4800F0B7FB03469AB20E4BD5
:10243C001A800E4B1B78002B02D00D4B01221A7008
:10244C000C4B1B7883F00103DBB2002B04D0064B42
:10245C001B889AB2084B1A80024800F0A9FB00BFF7
:10246C0080BD00BF1C060020000A0020D008002000
:10247C00D4080020F8090020F609002080B500AF30
:10248C00024802F007FC00BF80BD00BFA40600207C
:10249C0080B500AF4FF4805001F04CF900BF80BD07
:1024AC0080B586B000AF7860144A154BD31A7B61A7
:1024BC007B693B61134B1B68002B02D1114B124AF9
:1024CC001A60104B1A687B6813443A699A4207D217
:1024DC0004F09AFA03460C221A604FF0FF3309E01D
:1024EC00084B1B68FB60074B1A687B681344054A52
:1024FC001360FB6818461837BD4680BD005000209D
:10250C0000040000040A0020700A002080B400AF10
:10251C0000BFBD4680BC70470C480D490D4A0023D6
:10252C0002E0D458C4500433C4188C42F9D30A4A7C
:10253C000A4C002301E013600432A242FBD3FFF7E4
:10254C00E5FF04F067FAFEF7DFFC7047000000209F
:10255C00C8000020347B0008C80000206C0A002052
:10256C00FEE7000080B500AF084B1B68074A43F03C
:10257C0010031360032000F059FE002000F008F84F
:10258C00FFF776FD0023184680BD00BF00200240F7
:10259C0080B582B000AF7860124B1A68124B1B7872
:1025AC0019464FF47A73B3FBF1F3B2FBF3F318460D
:1025BC0000F071FE0346002B01D001230EE07B6876
:1025CC000F2B0AD8002279684FF0FF3000F039FE4B
:1025DC00064A7B681360002300E001231846083785
:1025EC00BD4680BD58000020600000205C0000202B
:1025FC0080B400AF054B1B781A46054B1B6813447F
:10260C00034A136000BFBD4680BC704760000020C9
:10261C00080A002080B400AF024B1B681846BD4668
:10262C0080BC7047080A002080B584B000AF786089
:10263C00FFF7F0FFB8607B68FB60FB68B3F1FF3F0E
:10264C0005D00A4B1B781A46FB681344FB6000BF8D
:10265C00FFF7E0FF0246BB68D31AFA689A42F7D834
:10266C0000BF00BF1037BD4680BD00BF600000201A
:10267C0080B586B000AF78600023FB7500233B610A
:10268C000023BB600023FB607B68002B01D101237E
:10269C00BEE07B689B68002B7B689B6A002B09D192
:1026AC007B680022DA627B68002283F82420786839
:1026BC00FFF710FD786800F0A3FC0346FB757B6800
:1026CC009B6A03F01003002B40F09980FB7D002BDC
:1026DC0040F095807B689B6A23F4885323F00203B7
:1026EC0043F002027B689A627B685A687B68DB69FC
:1026FC001A437B681B7B5B001343BA681343BB60B4
:10270C007B689B68B3F5807F03D07B689B68012B4B
:10271C0002D14FF4807300E000233A6913433B610C
:10272C007B681B7D012B19D17B681B7B002B09D18E
:10273C007B689B69013B5A033B69134343F4006379
:10274C003B610BE07B689B6A43F020027B689A62DA
:10275C007B68DB6A43F001027B68DA627B681B688A
:10276C005B6823F469417B681B683A690A435A60C9
:10277C007B681B689A68284B13407A681268B968A2
:10278C000B4393607B689B68B3F5807F03D07B68B9
:10279C009B68012B04D17B681B69013B1B05FB600B
:1027AC007B681B68DB6A23F470017B681B68FA6822
:1027BC000A43DA627B681B689A68184B1340BA6844
:1027CC009A420BD17B680022DA627B689B6A23F009
:1027DC00030343F001027B689A6218E07B689B6AF2
:1027EC0023F0120343F010027B689A627B68DB6A69
:1027FC0043F001027B68DA620123FB7507E07B681A
:10280C009B6A43F010027B689A620123FB75FB7D87
:10281C0018461837BD4680BDFDF7E1FFFE0E1FFFC1
:10282C0090B587B000AF7860396000237B610023DE
:10283C00FB6000233B61FFF7EDFE78617B681B6852
:10284C009B6803F48073002B0BD07B689B6A43F06E
:10285C0020027B689A627B68002283F82420012383
:10286C00D3E07B681B685B6803F48073002B31D169
:10287C007B681B68DB6A03F47003002B2AD121E010
:10288C003B68B3F1FF3F1DD03B68002B07D0FFF72F
:10289C00C1FE02467B69D31A3A689A4212D27B680F
:1028AC001B681B6803F00203002B0BD17B689B6A2F
:1028BC0043F004027B689A627B68002283F8242030
:1028CC000323A2E07B681B681B6803F00203002B48
:1028DC00D6D070E04F4B1C68022001F013FC03466D
:1028EC00B4FBF3F27B681B6819694B4B0B40002B54
:1028FC0018D17B681B68D968484B0B40002B11D151
:10290C007B681B681969464B0B40002B08D17B6810
:10291C001B68D968434B0B40002B01D1142320E0DA
:10292C0029231EE07B681B6819693D4B0B40002B6B
:10293C0006D17B681B68D9683A4B0B40002B0DD035
:10294C007B681B681969384B0B40002B08D17B68DE
:10295C001B68D968344B0B40002B01D1542300E089
:10296C00FC2302FB03F33B6121E03B68B3F1FF3F27
:10297C001AD03B68002B07D0FFF74CFE02467B6950
:10298C00D31A3A689A420FD2FB683A699A420BD929
:10299C007B689B6A43F004027B689A627B68002226
:1029AC0083F82420032330E0FB680133FB60FB68D1
:1029BC003A699A42D9D87B681B686FF012021A6088
:1029CC007B689B6A43F400727B689A627B681B6825
:1029DC009B6803F46023B3F5602F15D17B681B7BD8
:1029EC00002B11D17B689B6A23F480727B689A62FE
:1029FC007B689B6A03F48053002B05D17B689B6A30
:102A0C0043F001027B689A62002318461C37BD46CE
:102A1C0090BD00BF58000020244992242449920004
:102A2C0092244912922449004992240080B584B022
:102A3C0000AF78600023FB737B6893F82430012B84
:102A4C0001D10223A0E07B68012283F8242078685E
:102A5C0000F07CFA0346FB73FB7B002B40F08F806D
:102A6C007B689B6A23F4706323F0010343F4807248
:102A7C007B689A627B681B68454A934205D1454B3B
:102A8C005B6803F47023002B15D17B689B6A23F4DD
:102A9C0080127B689A627B681B685B6803F48063B6
:102AAC00002B26D07B689B6A23F4405343F480525E
:102ABC007B689A621DE07B689B6A43F480127B689A
:102ACC009A627B681B68334A934204D07B681B680C
:102ADC002F4A93420DD12F4B5B6803F48063002B7C
:102AEC0007D07B689B6A23F4405343F480527B6885
:102AFC009A627B689B6A03F48053002B06D07B6838
:102B0C00DB6A23F006027B68DA6202E07B68002253
:102B1C00DA627B68002283F824207B681B686FF0E4
:102B2C0002021A607B681B685A687B681B6842F05B
:102B3C0020025A607B681B689B6803F46023B3F522
:102B4C00602F13D17B681B68114A934205D1114B3E
:102B5C005B6803F47023002B08D17B681B689A68B0
:102B6C007B681B6842F4A0029A600CE07B681B68CF
:102B7C009A687B681B6842F480129A6003E07B6859
:102B8C00002283F82420FB7B18461037BD4680BDFD
:102B9C00002801400024014080B483B000AF78606D
:102BAC007B681B68DB6C18460C37BD4680BC7047D5
:102BBC0080B582B000AF78607B681B685B6803F0FF
:102BCC002003202B40D17B681B681B6803F0020399
:102BDC00022B39D17B689B6A03F01003002B05D1C3
:102BEC007B689B6A43F400727B689A627B681B6803
:102BFC009B6803F46023B3F5602F1DD17B681B7BAE
:102C0C00002B19D17B681B685A687B681B6822F003
:102C1C0020025A607B689B6A23F480727B689A62FC
:102C2C007B689B6A03F48053002B05D17B689B6AFD
:102C3C0043F001027B689A62786800F07CF87B684C
:102C4C001B686FF012021A607B681B685B6803F0EC
:102C5C008003802B4FD17B681B681B6803F0040337
:102C6C00042B48D17B689B6A03F01003002B05D121
:102C7C007B689B6A43F400527B689A627B681B6892
:102C8C009B6803F4E043B3F5E04F12D07B681B68FC
:102C9C005B6803F48063002B25D17B681B689B6801
:102CAC0003F46023B3F5602F1DD17B681B7B002BD5
:102CBC0019D17B681B685A687B681B6822F08002FC
:102CCC005A607B689B6A23F480527B689A627B68AB
:102CDC009B6A03F48073002B05D17B689B6A43F0DD
:102CEC0001027B689A62786800F0CBF97B681B68FC
:102CFC006FF00C021A607B681B685B6803F0400382
:102D0C00402B14D17B681B681B6803F00103012B5B
:102D1C000DD17B689B6A43F480327B689A62786839
:102D2C0000F012F87B681B686FF001021A6000BF9C
:102D3C000837BD4680BD80B483B000AF786000BF5B
:102D4C000C37BD4680BC704780B483B000AF786050
:102D5C0000BF0C37BD4680BC7047000080B485B006
:102D6C0000AF786039600023FB730023BB607B6885
:102D7C0093F82430012B01D10223DCE07B68012283
:102D8C0083F824203B685B68062B1CD87B681B6887
:102D9C00596B3B685A6813469B001344053B1F2232
:102DAC0002FA03F3DB4319403B6818683B685A6826
:102DBC0013469B001344053B00FA03F27B681B6827
:102DCC000A435A633CE03B685B680C2B1CD87B685D
:102DDC001B68196B3B685A6813469B001344233BD2
:102DEC001F2202FA03F3DB4319403B6818683B6867
:102DFC005A6813469B001344233B00FA03F27B688A
:102E0C001B680A431A631BE07B681B68D96A3B6822
:102E1C005A6813469B001344413B1F2202FA03F3EA
:102E2C00DB4319403B6818683B685A6813469B00A3
:102E3C001344413B00FA03F27B681B680A43DA62D5
:102E4C003B681B68092B1CD97B681B68D9683B68DD
:102E5C001A6813465B0013441E3B072202FA03F365
:102E6C00DB4319403B6898683B681A6813465B0063
:102E7C0013441E3B00FA03F27B681B680A43DA60BA
:102E8C0019E07B681B6819693B681A6813465B007C
:102E9C001344072202FA03F3DB4319403B6898689A
:102EAC003B681A6813465B00134400FA03F27B6814
:102EBC001B680A431A613B681B68102B03D03B68E4
:102ECC001B68112B32D17B681B681D4A934225D19C
:102EDC007B681B689B6803F40003002B26D17B687E
:102EEC001B689A687B681B6842F400029A603B6816
:102EFC001B68102B1AD1134B1B68134AA2FB03231C
:102F0C009A0C13469B0013445B00BB6002E0BB6849
:102F1C00013BBB60BB68002BF9D107E07B689B6A67
:102F2C0043F020027B689A620123FB737B680022CA
:102F3C0083F82420FB7B18461437BD4680BC7047B1
:102F4C00002401405800002083DE1B4380B584B070
:102F5C0000AF78600023FB600023BB607B681B68BC
:102F6C009B6803F00103012B40D07B681B689A68B7
:102F7C007B681B6842F001029A601F4B1B681F4A5A
:102F8C00A2FB03239B0CBB6002E0BB68013BBB6054
:102F9C00BB68002BF9D1FFF73DFBF8601FE0FFF792
:102FAC0039FB0246FB68D31A022B18D97B681B68C5
:102FBC009B6803F00103012B11D07B689B6A43F0E3
:102FCC0010027B689A627B68DB6A43F001027B68C3
:102FDC00DA627B68002283F82420012307E07B68F7
:102FEC001B689B6803F00103012BD8D10023184602
:102FFC001037BD4680BD00BF5800002083DE1B4348
:10300C0080B584B000AF78600023FB607B681B68E0
:10301C009B6803F00103012B2ED17B681B689A6817
:10302C007B681B6822F001029A60FFF7F3FAF860E4
:10303C001BE0FFF7EFFA0246FB68D31A022B14D9F8
:10304C007B681B689B6803F00103012B0DD17B6827
:10305C009B6A43F010027B689A627B68DB6A43F0E0
:10306C0001027B68DA62012307E07B681B689B68BE
:10307C0003F00103012BDCD0002318461037BD46AA
:10308C0080BD80B483B000AF786000BF0C37BD4604
:10309C0080BC704780B485B000AF78607B6803F06B
:1030AC000703FB600C4BDB68BB60BA684FF6FF0391
:1030BC001340BB60FB681A02BB68134343F0BF6349
:1030CC0043F40033BB60044ABB68D36000BF1437C1
:1030DC00BD4680BC704700BF00ED00E080B400AF7F
:1030EC00044BDB681B0A03F007031846BD4680BC83
:1030FC00704700BF00ED00E080B483B000AF034622
:10310C00FB7197F90730002B0BDBFB7903F01F02E7
:10311C00064997F907305B09012000FA02F241F8E1
:10312C00232000BF0C37BD4680BC704700E100E097
:10313C0080B483B000AF03463960FB7197F9073058
:10314C00002B0ADB3B68DAB20C4997F90730120105
:10315C00D2B20B4483F800230AE03B68DAB2084988
:10316C00FB7903F00F03043B1201D2B20B441A7625
:10317C0000BF0C37BD4680BC704700BF00E100E0CB
:10318C0000ED00E080B489B000AFF860B9607A60FF
:10319C00FB6803F00703FB61FB69C3F10703042B16
:1031AC0028BF0423BB61FB690433062B02D9FB69DE
:1031BC00033B00E000237B614FF0FF32BB6902FA56
:1031CC0003F3DA43BB681A407B699A404FF0FF3136
:1031DC007B6901FA03F3D9437B680B401343184610
:1031EC002437BD4680BC704780B582B000AF786094
:1031FC007B68013BB3F1807F01D301230FE00A4AC6
:10320C007B68013B53600F214FF0FF30FFF790FFBD
:10321C00054B00229A60044B07221A6000231846C3
:10322C000837BD4680BD00BF10E000E080B582B01D
:10323C0000AF78607868FFF72DFF00BF0837BD46F8
:10324C0080BD80B586B000AF0346B9607A60FB7371
:10325C0000237B61FFF742FF78617A68B96878696F
:10326C00FFF790FF024697F90F3011461846FFF70B
:10327C005FFF00BF1837BD4680BD80B582B000AF80
:10328C000346FB7197F907301846FFF735FF00BF6F
:10329C000837BD4680BD80B582B000AF78607868D5
:1032AC00FFF7A2FF034618460837BD4680BD000055
:1032BC0080B584B000AF78600023FB737B6893F813
:1032CC002130022B05D07B6804229A630123FB7307
:1032DC0051E07B681B681A687B681B6822F00E0241
:1032EC001A607B681B681A687B681B6822F00102F5
:1032FC001A607B681B68224A934229D07B681B6842
:10330C00204A934222D07B681B681F4A93421AD0F2
:10331C007B681B681D4A934212D07B681B681C4A51
:10332C0093420AD07B681B681A4A934202D14FF42D
:10333C0080130EE04FF080730BE04FF4803308E005
:10334C004FF4805305E04FF4807302E0102300E04B
:10335C000123114A53607B68012283F821207B688A
:10336C00002283F820207B685B6B002B03D07B68EA
:10337C005B6B78689847FB7B18461037BD4680BD61
:10338C00080002401C000240300002404400024091
:10339C00580002406C0002400000024080B48BB028
:1033AC0000AF7860396000237B6200233B6269E1E7
:1033BC0001227B6A02FA03F3FB613B681B68FA6922
:1033CC001340BB61BA69FB699A4240F058813B6873
:1033DC005B689A4A93425ED0984A934275D8984A51
:1033EC00934258D0964A93426FD8964A934252D001
:1033FC00944A934269D8944A93424CD0924A93424D
:10340C0063D8924A934246D0904A93425DD8122B8D
:10341C002AD8122B59D801A252F823F0A334000851
:10342C007D3400088F340008D1340008D7340008EC
:10343C00D7340008D7340008D7340008D734000834
:10344C00D7340008D7340008D7340008D734000824
:10345C00D7340008D7340008D7340008D734000814
:10346C008534000899340008794A934213D02CE033
:10347C003B68DB683B6229E03B68DB6804333B62FA
:10348C0024E03B68DB6808333B621FE03B68DB6889
:10349C000C333B621AE03B689B68002B02D104237F
:1034AC003B6213E03B689B68012B05D108233B6210
:1034BC007B68FA691A6109E008233B627B68FA6948
:1034CC005A6103E000233B6200E000BFBB69FF2BA5
:1034DC0001D87B6801E07B6804337B61BB69FF2BFF
:1034EC0002D87B6A9B0002E07B6A083B9B003B6135
:1034FC007B691A680F213B6901FA03F3DB431A401D
:10350C00396A3B6901FA03F31A437B691A603B6819
:10351C005B6803F08053002B00F0B1804D4B9B692E
:10352C004C4A43F0010393614A4B9B6903F001033E
:10353C00BB60BB68484A7B6A9B08023352F8233055
:10354C00FB607B6A03F003039B000F2202FA03F378
:10355C00DB43FA681340FB607B68404A934213D00C
:10356C007B683F4A93420DD07B683E4A934207D01A
:10357C007B683D4A934201D1032306E0042304E017
:10358C00022302E0012300E000237A6A02F0030226
:10359C0092009340FA681343FB602F497B6A9B08A7
:1035AC000233FA6841F823203B685B6803F48033EC
:1035BC00002B06D02D4B1A682C49BB6913430B60AA
:1035CC0006E02A4B1A68BB69DB43284913400B60A1
:1035DC003B685B6803F40033002B06D0234B5A681E
:1035EC002249BB6913434B6006E0204B5A68BB6908
:1035FC00DB431E4913404B603B685B6803F480134C
:10360C00002B06D0194B9A681849BB6913438B6081
:10361C0006E0164B9A68BB69DB43144913408B6078
:10362C003B685B6803F40013002B21D00F4BDA6866
:10363C000E49BB691343CB6021E000BF0000321080
:10364C0000003110000022100000211000001210A8
:10365C000000111000100240000001400008014061
:10366C00000C014000100140001401400004014016
:10367C000B4BDA68BB69DB4309491340CB607B6AAF
:10368C0001337B623B681A687B6A22FA03F3002BD6
:10369C007FF48EAE00BF00BF2C37BD4680BC704798
:1036AC000004014080B485B000AF78600B467B808D
:1036BC007B689A687B881340002B02D00123FB7334
:1036CC0001E00023FB73FB7B18461437BD4680BC1E
:1036DC00704780B483B000AF78600B467B80134694
:1036EC007B707B78002B03D07A887B681A6103E0AF
:1036FC007B881A047B681A6100BF0C37BD4680BCFE
:10370C00704780B485B000AF78600B467B807B68D7
:10371C00DB68FB607A88FB6813401A04FB68D943AA
:10372C007B880B401A437B681A6100BF1437BD4677
:10373C0080BC704780B582B000AF0346FB80084B5D
:10374C005A69FB881340002B06D0054AFB8853614D
:10375C00FB881846FDF7D6FA00BF0837BD4680BD7A
:10376C000004014080B586B000AF78607B68002B08
:10377C0001D1012372E27B681B6803F00103002B6B
:10378C0000F08780924B5B6803F00C03042B0CD089
:10379C008F4B5B6803F00C03082B12D18C4B5B68CE
:1037AC0003F48033B3F5803F0BD1894B1B6803F4D2
:1037BC000033002B6CD07B685B68002B68D1012335
:1037CC004CE27B685B68B3F5803F06D1804B1B688D
:1037DC007F4A43F4803313602EE07B685B68002BD8
:1037EC000CD17B4B1B687A4A23F480331360784BE3
:1037FC001B68774A23F4802313601DE07B685B68A9
:10380C00B3F5A02F0CD1724B1B68714A43F4802383
:10381C0013606F4B1B686E4A43F4803313600BE0EC
:10382C006B4B1B686A4A23F480331360684B1B682C
:10383C00674A23F4802313607B685B68002B13D0EA
:10384C00FEF7E8FE386108E0FEF7E4FE02463B694D
:10385C00D31A642B01D9032300E25D4B1B6803F4DC
:10386C000033002BF0D014E0FEF7D4FE386108E0F2
:10387C00FEF7D0FE02463B69D31A642B01D9032311
:10388C00ECE1534B1B6803F40033002BF0D100E048
:10389C0000BF7B681B6803F00203002B63D04C4B0A
:1038AC005B6803F00C03002B0BD0494B5B6803F0F7
:1038BC000C03082B1CD1464B5B6803F48033002BA4
:1038CC0016D1434B1B6803F00203002B05D07B6819
:1038DC001B69012B01D00123C0E13D4B1B6823F078
:1038EC00F8027B685B69DB00394913430B603AE0F3
:1038FC007B681B69002B20D0364B01221A60FEF727
:10390C0089FE386108E0FEF785FE02463B69D31A52
:10391C00022B01D90323A1E12D4B1B6803F00203F9
:10392C00002BF0D02A4B1B6823F0F8027B685B69F4
:10393C00DB00274913430B6015E0264B00221A606D
:10394C00FEF768FE386108E0FEF764FE02463B694C
:10395C00D31A022B01D9032380E11D4B1B6803F002
:10396C000203002BF0D17B681B6803F00803002BCB
:10397C003AD07B689B69002B19D0174B01221A6037
:10398C00FEF748FE386108E0FEF744FE02463B694C
:10399C00D31A022B01D9032360E10D4B5B6A03F0B0
:1039AC000203002BF0D0012000F0D8FA1CE00A4BE7
:1039BC0000221A60FEF72EFE38610FE0FEF72AFE99
:1039CC0002463B69D31A022B08D9032346E100BFF8
:1039DC00001002400000424280044242924B5B6A5B
:1039EC0003F00203002BE9D17B681B6803F004038E
:1039FC00002B00F0A6800023FB758B4BDB6903F0DA
:103A0C008053002B0DD1884BDB69874A43F08053E0
:103A1C00D361854BDB6903F08053BB60BB6801232A
:103A2C00FB75824B1B6803F48073002B18D17F4B02
:103A3C001B687E4A43F480731360FEF7EBFD38611C
:103A4C0008E0FEF7E7FD02463B69D31A642B01D967
:103A5C00032303E1754B1B6803F48073002BF0D038
:103A6C007B68DB68012B06D16F4B1B6A6E4A43F0F7
:103A7C00010313622DE07B68DB68002B0CD16A4BD1
:103A8C001B6A694A23F001031362674B1B6A664A7F
:103A9C0023F0040313621CE07B68DB68052B0CD15C
:103AAC00614B1B6A604A43F0040313625E4B1B6A52
:103ABC005D4A43F0010313620BE05B4B1B6A5A4AED
:103ACC0023F001031362584B1B6A574A23F004037B
:103ADC0013627B68DB68002B15D0FEF79BFD386109
:103AEC000AE0FEF797FD02463B69D31A41F2883291
:103AFC00934201D90323B1E04B4B1B6A03F0020341
:103B0C00002BEED014E0FEF785FD38610AE0FEF7DD
:103B1C0081FD02463B69D31A41F28832934201D9A6
:103B2C0003239BE0404B1B6A03F00203002BEED1F6
:103B3C00FB7D012B05D13C4BDB693B4A23F08053C9
:103B4C00D3617B68DB69002B00F08780364B5B68A8
:103B5C0003F00C03082B61D07B68DB69022B46D188
:103B6C00334B00221A60FEF755FD386108E0FEF772
:103B7C0051FD02463B69D31A022B01D903236DE098
:103B8C00294B1B6803F00073002BF0D17B681B6A78
:103B9C00B3F5803F08D1244B5B6823F400327B687B
:103BAC009B68214913434B601F4B5B6823F47412D1
:103BBC007B68196A7B685B6A0B431B4913434B6038
:103BCC001B4B01221A60FEF725FD386108E0FEF759
:103BDC0021FD02463B69D31A022B01D903233DE098
:103BEC00114B1B6803F00073002BF0D035E0104B29
:103BFC0000221A60FEF70EFD386108E0FEF70AFDA0
:103C0C0002463B69D31A022B01D9032326E0064B4B
:103C1C001B6803F00073002BF0D11EE07B68DB699E
:103C2C00012B07D1012319E0001002400070004065
:103C3C00600042420B4B5B68FB60FB6803F4803214
:103C4C007B681B6A9A4206D1FB6803F470127B688E
:103C5C005B6A9A4201D0012300E000231846183712
:103C6C00BD4680BD0010024080B584B000AF7860C6
:103C7C0039607B68002B01D10123D0E06A4B1B68B3
:103C8C0003F007033A689A4210D9674B1B6823F07C
:103C9C00070265493B6813430B60634B1B6803F0D9
:103CAC0007033A689A4201D00123B8E07B681B688D
:103CBC0003F00203002B20D07B681B6803F0040385
:103CCC00002B05D0594B5B68584A43F4E0635360B2
:103CDC007B681B6803F00803002B05D0534B5B6813
:103CEC00524A43F460535360504B5B6823F0F0022C
:103CFC007B689B684D4913434B607B681B6803F0E2
:103D0C000103002B40D07B685B68012B07D1474B2C
:103D1C001B6803F40033002B15D101237FE07B6873
:103D2C005B68022B07D1414B1B6803F00073002B1F
:103D3C0009D1012373E03D4B1B6803F00203002BF8
:103D4C0001D101236BE0394B5B6823F003027B68E4
:103D5C005B68364913434B60FEF75CFCF8600AE085
:103D6C00FEF758FC0246FB68D31A41F288329342A4
:103D7C0001D9032353E02D4B5B6803F00C027B68E5
:103D8C005B689B009A42EBD1274B1B6803F007033F
:103D9C003A689A4210D2244B1B6823F0070222493E
:103DAC003B6813430B60204B1B6803F007033A6816
:103DBC009A4201D0012332E07B681B6803F00403B4
:103DCC00002B08D0194B5B6823F4E0627B68DB683E
:103DDC00164913434B607B681B6803F00803002BE8
:103DEC0009D0124B5B6823F460527B681B69DB00C3
:103DFC000E4913434B6000F021F802460B4B5B68F5
:103E0C001B0903F00F030A49CB5C22FA03F3094A9E
:103E1C001360094B1B681846FEF7BAFB00231846C3
:103E2C001037BD4680BD00BF00200240001002408C
:103E3C00E07A0008580000205C00002090B48AB0A2
:103E4C0000AF294B3C1D0FCB84E80F0040F201233F
:103E5C003B800023FB610023BB6100237B620023BA
:103E6C007B6100233B62214B5B68FB61FB6903F0C8
:103E7C000C03042B02D0082B03D02BE01C4B3B6211
:103E8C002BE0FB699B0C03F00F0328333B4413F826
:103E9C00243C7B61FB6903F48033002B12D0134B61
:103EAC005B685B0C03F0010328333B4413F8283C9C
:103EBC00BB617B690E4A03FB02F2BB69B2FBF3F3F5
:103ECC007B6204E07B690B4A02FB03F37B627B6A37
:103EDC003B6202E0064B3B6200BF3B6A1846283748
:103EEC00BD4690BC704700BF8473000800100240B0
:103EFC0000127A0000093D0080B400AF024B1B6831
:103F0C001846BD4680BC70475800002080B500AFF5
:103F1C00FFF7F2FF0246054B5B681B0A03F0070331
:103F2C000349CB5C22FA03F3184680BD0010024013
:103F3C00F07A000880B500AFFFF7DEFF0246054BB4
:103F4C005B68DB0A03F007030349CB5C22FA03F33B
:103F5C00184680BD00100240F07A000880B485B08D
:103F6C0000AF78600A4B1B680A4AA2FB03235B0A6A
:103F7C007A6802FB03F3FB6000BFFB685A1EFA6011
:103F8C00002BF9D100BF00BF1437BD4680BC704771
:103F9C0058000020D34D621080B586B000AF786019
:103FAC0000233B610023FB607B681B6803F001036B
:103FBC00002B7DD00023FB754F4BDB6903F0805346
:103FCC00002B0DD14C4BDB694B4A43F08053D36132
:103FDC00494BDB6903F08053BB60BB680123FB7565
:103FEC00464B1B6803F48073002B18D1434B1B68A2
:103FFC00424A43F480731360FEF70CFB386108E00F
:10400C00FEF708FB02463B69D31A642B01D9032344
:10401C006DE03A4B1B6803F48073002BF0D0364BE9
:10402C001B6A03F44073FB60FB68002B2ED07B688B
:10403C005B6803F44073FA689A4227D02E4B1B6AD4
:10404C0023F44073FB602E4B01221A602C4B002290
:10405C001A60294AFB681362FB6803F00103002B0A
:10406C0014D0FEF7D7FA38610AE0FEF7D3FA02460D
:10407C003B69D31A41F28832934201D9032336E0CB
:10408C001D4B1B6A03F00203002BEED01A4B1B6A6C
:10409C0023F440727B685B68174913430B62FB7D0A
:1040AC00012B05D1144BDB69134A23F08053D361E8
:1040BC007B681B6803F00203002B08D00E4B5B6877
:1040CC0023F440427B689B680B4913434B607B682D
:1040DC001B6803F01003002B08D0074B5B6823F41C
:1040EC0080027B68DB68044913434B60002318464D
:1040FC001837BD4680BD00BF001002400070004064
:10410C004004424290B58DB000AF7860584B07F137
:10411C000C040FCB84E80F0040F201233B810023F9
:10412C007B620023FB6200233B620023FB610023C4
:10413C00BB627B68102B0AD07B68102B00F28E8040
:10414C007B68012B49D07B68022B79D086E0494BE8
:10415C005B68FB61474B1B6803F08073002B7FD0BF
:10416C00FB699B0C03F00F0330333B4413F8243CE6
:10417C003B62FB6903F48033002B17D03D4B5B682B
:10418C005B0C03F0010330333B4413F8283C7B6297
:10419C00FB6903F48033002B0DD0374A7B6AB2FBEA
:1041AC00F3F23B6A02FB03F3FB6204E03B6A334A23
:1041BC0002FB03F3FB622F4B5B6803F48003B3F544
:1041CC00800F02D1FB6ABB624AE0FB6A5B002C4A9F
:1041DC00A2FB03235B08BB6242E0264B1B6AFB611C
:1041EC00FB6903F44073B3F5807F08D1FB6903F0DE
:1041FC000203002B03D04FF40043BB621FE0FB69AA
:10420C0003F44073B3F5007F09D11A4B5B6A03F0DA
:10421C000203002B03D049F64043BB620FE0FB695D
:10422C0003F44073B3F5407F1CD1124B1B6803F4AD
:10423C000033002B16D04FF22443BB6212E011E086
:10424C00FFF778FE02460B4B5B689B0B03F00303F6
:10425C0001335B00B2FBF3F3BB6204E000BF02E08E
:10426C0000BF00E000BFBB6A18463437BD4690BDA6
:10427C00947300080010024000127A0000093D00FF
:10428C00ABAAAAAA80B582B000AF78607B68002B7D
:10429C0001D1012376E07B685B6A002B08D17B6837
:1042AC005B68B3F5827F09D07B680022DA6105E098
:1042BC007B6800221A617B6800225A617B680022AD
:1042CC009A627B6893F85130DBB2002B06D17B6885
:1042DC00002283F850207868FDF740FF7B680222AB
:1042EC0083F851207B681B681A687B681B6822F076
:1042FC0040021A607B685B6803F482727B689B687F
:10430C0003F404431A437B68DB6803F400631A4329
:10431C007B681B6903F002031A437B685B6903F03B
:10432C0001031A437B689B6903F400731A437B688F
:10433C00DB6903F038031A437B681B6A03F08003C4
:10434C0042EA03017B689B6A03F400527B681B689A
:10435C000A431A607B689B691A0C7B681B6802F025
:10436C0004025A607B681B68DA697B681B6822F45C
:10437C000062DA617B6800225A657B68012283F84F
:10438C005120002318460837BD4680BD80B588B043
:10439C0000AFF860B9603B601346FB800023FB77ED
:1043AC00FB6893F85030012B01D1022326E1FB6806
:1043BC00012283F85020FEF72DF9B861FB88FB82AF
:1043CC00FB6893F85130DBB2012B02D00223FB7750
:1043DC000BE1BB68002B02D0FB88002B02D1012320
:1043EC00FB7702E1FB68032283F85120FB68002273
:1043FC005A65FB68BA681A63FB68FA889A86FB6888
:10440C00FA88DA86FB6800229A63FB6800229A8796
:10441C00FB680022DA87FB6800225A64FB680022E2
:10442C001A64FB689B68B3F5004F0FD1FB681B68DF
:10443C001A68FB681B6822F040021A60FB681B6854
:10444C001A68FB681B6842F480421A60FB681B68A0
:10445C001B6803F04003402B07D0FB681B681A68ED
:10446C00FB681B6842F040021A60FB68DB68B3F51E
:10447C00006F4BD1FB685B68002B02D0FB8A012BD1
:10448C003ED1FB681B6B1A88FB681B68DA60FB6803
:10449C001B6B9A1CFB681A63FB68DB8E9BB2013B9F
:1044AC009AB2FB68DA862BE0FB681B689B6803F00A
:1044BC000203022B12D1FB681B6B1A88FB681B686A
:1044CC00DA60FB681B6B9A1CFB681A63FB68DB8E5B
:1044DC009BB2013B9AB2FB68DA8611E0FEF79AF8C0
:1044EC000246BB69D31A3A689A4203D83B68B3F1C7
:1044FC00FF3F02D13B68002B02D10323FB7774E012
:10450C00FB68DB8E9BB2002BCED14CE0FB685B686A
:10451C00002B02D0FB8A012B40D1FB681A6BFB6885
:10452C001B680C3312781A70FB681B6B5A1CFB68E7
:10453C001A63FB68DB8E9BB2013B9AB2FB68DA868E
:10454C002CE0FB681B689B6803F00203022B13D161
:10455C00FB681A6BFB681B680C3312781A70FB68CB
:10456C001B6B5A1CFB681A63FB68DB8E9BB2013B0E
:10457C009AB2FB68DA8611E0FEF74CF80246BB698A
:10458C00D31A3A689A4203D83B68B3F1FF3F02D181
:10459C003B68002B02D10323FB7726E0FB68DB8E04
:1045AC009BB2002BCDD1BA693968F86800F01AFEBD
:1045BC000346002B02D0FB6820225A65FB689B68DF
:1045CC00002B0AD100233B61FB681B68DB683B6155
:1045DC00FB681B689B683B613B69FB685B6D002B50
:1045EC0002D00123FB7700E000BFFB68012283F8B7
:1045FC005120FB68002283F85020FB7F184620379F
:10460C00BD4680BD80B588B002AFF860B9603B6034
:10461C001346FB800023FB75FB685B68B3F5827F58
:10462C0012D1FB689B68002B0ED1FB68042283F827
:10463C005120FA883B6800931346BA68B968F86849
:10464C0000F0F1F80346EAE0FB6893F85030012BD8
:10465C0001D10223E3E0FB68012283F85020FDF72F
:10466C00D9FF3861FB6893F85130DBB2012B02D0D3
:10467C000223FB75CAE0BB68002B02D0FB88002B21
:10468C0002D10123FB75C1E0FB68042283F85120A1
:10469C00FB6800225A65FB68BA689A63FB68FA8863
:1046AC009A87FB68FA88DA87FB6800221A63FB6832
:1046BC0000229A86FB680022DA86FB6800221A64C4
:1046CC00FB6800225A64FB689B68B3F5004F0FD15E
:1046DC00FB681B681A68FB681B6822F040021A60B2
:1046EC00FB681B681A68FB681B6822F480421A601E
:1046FC00FB681B681B6803F04003402B07D0FB686A
:10470C001B681A68FB681B6842F040021A60FB6861
:10471C00DB68002B62D12EE0FB681B689B6803F002
:10472C000103012B15D1FB681B6803F10C02FB681C
:10473C009B6B1278D2B21A70FB689B6B5A1CFB688D
:10474C009A63FB68DB8F9BB2013B9AB2FB68DA87FA
:10475C0011E0FDF75FFF02463B69D31A3A689A42B3
:10476C0003D83B68B3F1FF3F02D13B68002B02D169
:10477C000323FB754AE0FB68DB8F9BB2002BCBD18C
:10478C0031E0FB681B689B6803F00103012B13D11C
:10479C00FB681B68DA68FB689B6B92B21A80FB683B
:1047AC009B6B9A1CFB689A63FB68DB8F9BB2013B8B
:1047BC009AB2FB68DA8711E0FDF72CFF02463B69E1
:1047CC00D31A3A689A4203D83B68B3F1FF3F02D13F
:1047DC003B68002B02D10323FB7517E0FB68DB8FD2
:1047EC009BB2002BCDD13A693968F86800F0A8FC6F
:1047FC000346002B02D0FB6820225A65FB685B6DD8
:10480C00002B02D00123FB7500E000BFFB680122E6
:10481C0083F85120FB68002283F85020FB7D18465A
:10482C001837BD4680BD80B58CB000AFF860B9605C
:10483C007A607B800123FB62002387F82B30FB68B6
:10484C0093F85030012B01D102238AE1FB6801223D
:10485C0083F85020FDF7DEFE7862FB6893F8513048
:10486C0087F82330FB685B68FB617B887B8397F858
:10487C002330012B0FD0FB69B3F5827F07D1FB6886
:10488C009B68002B03D197F82330042B03D0022311
:10489C0087F82B305BE1BB68002B05D07B68002BC5
:1048AC0002D07B88002B03D1012387F82B304EE1FB
:1048BC00FB6893F85130DBB2042B03D0FB68052264
:1048CC0083F85120FB6800225A65FB687A689A636A
:1048DC00FB687A88DA87FB687A889A87FB68BA68FB
:1048EC001A63FB687A88DA86FB687A889A86FB6892
:1048FC0000221A64FB6800225A64FB681B681B6860
:10490C0003F04003402B07D0FB681B681A68FB6858
:10491C001B6842F040021A60FB68DB68B3F5006F5D
:10492C0078D1FB685B68002B02D07B8B012B66D1A6
:10493C00FB681B6B1A88FB681B68DA60FB681B6BD7
:10494C009A1CFB681A63FB68DB8E9BB2013B9AB224
:10495C00FB68DA8653E0FB681B689B6803F0020374
:10496C00022B1BD1FB68DB8E9BB2002B16D0FB6A93
:10497C00012B13D1FB681B6B1A88FB681B68DA6070
:10498C00FB681B6B9A1CFB681A63FB68DB8E9BB283
:10499C00013B9AB2FB68DA860023FB62FB681B685A
:1049AC009B6803F00103012B19D1FB68DB8F9BB2D1
:1049BC00002B14D0FB681B68DA68FB689B6B92B207
:1049CC001A80FB689B6B9A1CFB689A63FB68DB8FF5
:1049DC009BB2013B9AB2FB68DA870123FB62FDF7BD
:1049EC0019FE02467B6AD31ABA6B9A4207D8BB6B84
:1049FC00B3F1FF3F03D0032387F82B30A7E0FB680C
:104A0C00DB8E9BB2002BA6D1FB68DB8F9BB2002BFD
:104A1C00A1D17CE0FB685B68002B02D07B8B012B67
:104A2C006BD1FB681A6BFB681B680C3312781A701D
:104A3C00FB681B6B5A1CFB681A63FB68DB8E9BB212
:104A4C00013B9AB2FB68DA8657E0FB681B689B68EF
:104A5C0003F00203022B1CD1FB68DB8E9BB2002BF4
:104A6C0017D0FB6A012B14D1FB681A6BFB681B680F
:104A7C000C3312781A70FB681B6B5A1CFB681A6398
:104A8C00FB68DB8E9BB2013B9AB2FB68DA86002393
:104A9C00FB62FB681B689B6803F00103012B19D1B7
:104AAC00FB68DB8F9BB2002B14D0FB681B68DA68A9
:104ABC00FB689B6BD2B21A70FB689B6B5A1CFB6831
:104ACC009A63FB68DB8F9BB2013B9AB2FB68DA8777
:104ADC000123FB62FDF79EFD02467B6AD31ABA6B7B
:104AEC009A4203D8BB6BB3F1FF3F02D1BB6B002BD7
:104AFC0003D1032387F82B3029E0FB68DB8E9BB2B4
:104B0C00002BA2D1FB68DB8F9BB2002B9DD17A6A64
:104B1C00B96BF86800F066FB0346002B06D0012346
:104B2C0087F82B30FB6820225A6510E0FB689B68E5
:104B3C00002B0BD100237B61FB681B68DB687B615E
:104B4C00FB681B689B687B617B6900E000BFFB68AE
:104B5C00012283F85120FB68002283F8502097F83B
:104B6C002B3018463037BD4680BD000080B487B06E
:104B7C0000AFF860B9607A607B800023FB75FB683E
:104B8C0093F85030012B01D1022375E0FB68012210
:104B9C0083F85020FB6893F85130BB75FB685B6859
:104BAC003B61BB7D012B0DD03B69B3F5827F06D1F8
:104BBC00FB689B68002B02D1BB7D042B02D0022327
:104BCC00FB7554E0BB68002B05D07B68002B02D032
:104BDC007B88002B02D10123FB7548E0FB6893F81E
:104BEC005130DBB2042B03D0FB68052283F8512033
:104BFC00FB6800225A65FB68BA681A63FB687A88FE
:104C0C009A86FB687A88DA86FB687A689A63FB680E
:104C1C007A889A87FB687A88DA87FB68DB68002BCE
:104C2C0006D0FB68174A1A64FB68174A5A6405E0F9
:104C3C00FB68164A1A64FB68154A5A64FB681B68C1
:104C4C005A68FB681B6842F0E0025A60FB681B68FC
:104C5C001B6803F04003402B08D0FB681B681A68E4
:104C6C00FB681B6842F040021A6000E000BFFB6862
:104C7C00002283F85020FB7D18461C37BD4680BCB3
:104C8C00704700BF7D4F0008DD4F0008B94E00088B
:104C9C001D4F000880B588B000AF78607B681B683A
:104CAC005B68FB617B681B689B68BB61BB699B098C
:104CBC0003F00103002B0FD1BB6903F00103002BA0
:104CCC000AD0FB699B0903F00103002B04D07B681D
:104CDC001B6C78689847BEE0BB695B0803F0010366
:104CEC00002B0AD0FB69DB0903F00103002B04D075
:104CFC007B685B6C78689847ADE0BB695B0903F037
:104D0C000103002B06D1BB699B0903F00103002BA7
:104D1C0000F0A180FB695B0903F00103002B00F09C
:104D2C009A80BB699B0903F00103002B23D07B689D
:104D3C0093F85130DBB2032B11D07B685B6D43F0E1
:104D4C0004027B685A6500237B617B681B68DB6807
:104D5C007B617B681B689B687B617B690BE0002334
:104D6C003B617B681B68DB683B617B681B689B68ED
:104D7C003B613B696FE0BB695B0903F00103002BEE
:104D8C0014D07B685B6D43F001027B685A6500238D
:104D9C00FB607B681B689B68FB607B681B681A6800
:104DAC007B681B6822F040021A60FB687B685B6DB5
:104DBC00002B4FD07B681B685A687B681B6822F0FD
:104DCC00E0025A607B68012283F85120FB6903F0F2
:104DDC000203002B04D1FB6903F00103002B34D038
:104DEC007B681B685A687B681B6822F003025A6058
:104DFC007B68DB6C002B11D07B68DB6C174A5A6329
:104E0C007B68DB6C1846FEF753FA0346002B05D083
:104E1C007B685B6D43F040027B685A657B689B6CDA
:104E2C00002B16D07B689B6C0C4A5A637B689B6C7E
:104E3C001846FEF73DFA0346002B0AD07B685B6DE3
:104E4C0043F040027B685A6503E0786800F011F883
:104E5C0000E000BF00BF2037BD4680BD914E00086A
:104E6C0080B483B000AF786000BF0C37BD4680BC07
:104E7C00704780B483B000AF786000BF0C37BD467C
:104E8C0080BC704780B584B000AF78607B685B6A8B
:104E9C00FB60FB680022DA87FB680022DA86F86880
:104EAC00FFF7E7FF00BF1037BD4680BD80B582B06D
:104EBC0000AF78607B681B6803F10C027B689B6B0E
:104ECC001278D2B21A707B689B6B5A1C7B689A63FF
:104EDC007B68DB8F9BB2013B9AB27B68DA877B687D
:104EEC00DB8F9BB2002B0FD17B681B685A687B68E9
:104EFC001B6822F060025A607B68DB8E9BB2002B31
:104F0C0002D1786800F08CF900BF0837BD4680BD2F
:104F1C0080B582B000AF78607B681A6B7B681B68C9
:104F2C000C3312781A707B681B6B5A1C7B681A63E3
:104F3C007B68DB8E9BB2013B9AB27B68DA867B681E
:104F4C00DB8E9BB2002B0FD17B681B685A687B6889
:104F5C001B6822F080025A607B68DB8F9BB2002BAF
:104F6C0002D1786800F05CF900BF0837BD4680BDFF
:104F7C0080B582B000AF78607B681B68DA687B68AC
:104F8C009B6B92B21A807B689B6B9A1C7B689A63B2
:104F9C007B68DB8F9BB2013B9AB27B68DA877B68BC
:104FAC00DB8F9BB2002B0FD17B681B685A687B6828
:104FBC001B6822F040025A607B68DB8E9BB2002B90
:104FCC0002D1786800F02CF900BF0837BD4680BDCF
:104FDC0080B582B000AF78607B681B6B1A887B68E9
:104FEC001B68DA607B681B6B9A1C7B681A637B6896
:104FFC00DB8E9BB2013B9AB27B68DA867B68DB8ED8
:10500C009BB2002B0FD17B681B685A687B681B68AE
:10501C0022F080025A607B68DB8F9BB2002B02D19E
:10502C00786800F0FDF800BF0837BD4680BD000071
:10503C0080B588B000AFF860B9603B601346FB7177
:10504C00FDF7E8FA0246BB6A9B1A3A681344FB6107
:10505C00FDF7E0FAB861394B1B685B011B0DFA696F
:10506C0002FB03F37B6154E03B68B3F1FF3F50D08C
:10507C00FDF7D0FA0246BB69D31AFA699A4202D9F3
:10508C00FB69002B3DD1FB681B685A68FB681B68E9
:10509C0022F0E0025A60FB685B68B3F5827F11D1A5
:1050AC00FB689B68B3F5004F04D0FB689B68B3F5B5
:1050BC00806F07D1FB681B681A68FB681B6822F0BD
:1050CC0040021A60FB689B6AB3F5005F0FD1FB6866
:1050DC001B681A68FB681B6822F400521A60FB6894
:1050EC001B681A68FB681B6842F400521A60FB6864
:1050FC00012283F85120FB68002283F850200323FF
:10510C0017E07B69002B01D10023FB617B69013B1C
:10511C007B61FB681B689A68BB681340BA689A424B
:10512C000CBF01230023DBB21A46FB799A429BD1B8
:10513C00002318462037BD4680BD00BF5800002014
:10514C0080B586B002AFF860B9607A60FB685B68C6
:10515C00B3F5827F11D1FB689B68B3F5004F04D087
:10516C00FB689B68B3F5806F07D1FB681B681A68F6
:10517C00FB681B6822F040021A60FB685B68B3F5A1
:10518C00827F17D1FB689B68B3F5806F12D17B6867
:10519C000093BB6800220121F868FFF749FF034622
:1051AC00002B1AD0FB685B6D43F02002FB685A653C
:1051BC00032313E07B680093BB6800228021F8680E
:1051CC00FFF736FF0346002B07D0FB685B6D43F0FF
:1051DC002002FB685A65032300E0002318461037B1
:1051EC00BD4680BD80B586B002AFF860B9607A600C
:1051FC007B680093BB6800228021F868FFF718FFDA
:10520C000346002B07D0FB685B6D43F02002FB6864
:10521C005A65032300E0002318461037BD4680BDB5
:10522C0080B586B000AF7860354B1B68354AA2FB61
:10523C0003235B0A642202FB03F33B61FDF7EAF9EB
:10524C0078617B681B685A687B681B6822F02002B7
:10525C005A603B69002B06D17B685B6D43F02002E2
:10526C007B685A6509E03B69013B3B617B681B68C5
:10527C009B6803F00203002BEBD07A6964217868F9
:10528C00FFF7B0FF0346002B05D07B685B6D43F046
:10529C0020027B685A657B689B68002B0AD100232F
:1052AC00FB607B681B68DB68FB607B681B689B682A
:1052BC00FB60FB687B685B6D002B15D17B6893F8FA
:1052CC005130DBB2042B07D17B68012283F85120CB
:1052DC007868FFF7C5FD0EE07B68012283F851204A
:1052EC007868FBF7DDFD06E07B68012283F851202E
:1052FC007868FFF7BEFD00BF1837BD4680BD00BF04
:10530C0058000020F119760580B582B000AF7860A6
:10531C007B68002B01D1012341E07B6893F83D3081
:10532C00DBB2002B06D17B68002283F83C20786826
:10533C00FCF7A2FF7B68022283F83D207B681A6889
:10534C007B6804331946104600F002FB7B6801228F
:10535C0083F846207B68012283F83E207B6801227B
:10536C0083F83F207B68012283F840207B68012270
:10537C0083F841207B68012283F842207B6801225C
:10538C0083F843207B68012283F844207B68012248
:10539C0083F845207B68012283F83D2000231846C2
:1053AC000837BD4680BD000080B485B000AF786082
:1053BC007B6893F83D30DBB2012B01D0012332E046
:1053CC007B68022283F83D207B681B68184A934255
:1053DC000ED07B681B68B3F1804F09D07B681B68CB
:1053EC00144A934204D07B681B68134A934211D130
:1053FC007B681B689B6803F00703FB60FB68062B4C
:10540C0010D07B681B681A687B681B6842F001022D
:10541C001A6007E07B681B681A687B681B6842F09F
:10542C0001021A60002318461437BD4680BC704731
:10543C00002C0140000400400008004080B582B000
:10544C0000AF78607B68002B01D1012341E07B68C1
:10545C0093F83D30DBB2002B06D17B68002283F839
:10546C003C20786800F039F87B68022283F83D20F4
:10547C007B681A687B6804331946104600F068FA9A
:10548C007B68012283F846207B68012283F83E204A
:10549C007B68012283F83F207B68012283F840203F
:1054AC007B68012283F841207B68012283F842202B
:1054BC007B68012283F843207B68012283F8442017
:1054CC007B68012283F845207B68012283F83D200C
:1054DC00002318460837BD4680BD80B483B000AFAA
:1054EC00786000BF0C37BD4680BC704780B582B079
:1054FC0000AF786039607B68002B01D1012341E05B
:10550C007B6893F83D30DBB2002B06D17B68002220
:10551C0083F83C20786800F039F87B68022283F825
:10552C003D207B681A687B6804331946104600F0EE
:10553C000FFA7B681B681A687B681B6822F00802EC
:10554C001A607B681B6819687B681B683A680A4399
:10555C001A607B68012283F846207B68012283F85D
:10556C003E207B68012283F83F207B68012283F870
:10557C0042207B68012283F843207B68012283F858
:10558C003D20002318460837BD4680BD80B483B04B
:10559C0000AF786000BF0C37BD4680BC7047000080
:1055AC0080B584B000AF786039607B6893F83E308A
:1055BC00FB737B6893F83F30BB737B6893F8423086
:1055CC007B737B6893F843303B73FB7B012B08D1D7
:1055DC00BB7B012B05D17B7B012B02D13B7B012BB0
:1055EC0001D001232BE07B68022283F83E207B68EC
:1055FC00022283F83F207B68022283F842207B68DA
:10560C00022283F843207B681B6801220021184684
:10561C0000F01EFC7B681B6801220421184600F078
:10562C0017FC7B681B68084A934207D17B681B6890
:10563C005A6C7B681B6842F400425A64002318467B
:10564C001037BD4680BD00BF002C014080B584B032
:10565C0000AFF860B9607A60FB6893F83C30012BBE
:10566C0001D10223ACE0FB68012283F83C207B686B
:10567C000C2B00F29F8001A252F823F0BD560008BB
:10568C00C1570008C1570008C1570008FD56000853
:10569C00C1570008C1570008C15700083F57000800
:1056AC00C1570008C1570008C15700087F570008B0
:1056BC00FB681B68B968184600F0ACF9FB681B68FE
:1056CC009A69FB681B6842F008029A61FB681B68C8
:1056DC009A69FB681B6822F004029A61FB681B68DC
:1056EC009969BB681A69FB681B680A439A6162E096
:1056FC00FB681B68B968184600F0F2F9FB681B6878
:10570C009A69FB681B6842F400629A61FB681B682B
:10571C009A69FB681B6822F480629A61FB681B68BB
:10572C009969BB681B691A02FB681B680A439A617A
:10573C0041E0FB681B68B968184600F03BFAFB684F
:10574C001B68DA69FB681B6842F00802DA61FB68C7
:10575C001B68DA69FB681B6822F00402DA61FB68DB
:10576C001B68D969BB681A69FB681B680A43DA6154
:10577C0021E0FB681B68B968184600F085FAFB68E5
:10578C001B68DA69FB681B6842F40062DA61FB682B
:10579C001B68DA69FB681B6822F48062DA61FB68BB
:1057AC001B68D969BB681B691A02FB681B680A4332
:1057BC00DA6100E000BFFB68002283F83C20002384
:1057CC0018461037BD4680BD80B584B000AF7860F8
:1057DC0039607B6893F83C30012B01D10223B3E094
:1057EC007B68012283F83C207B68022283F83D20F1
:1057FC007B681B689B68FB60FB6823F07703FB608E
:10580C00FB6823F47F43FB607B681B68FA689A6033
:10581C003B681B68B3F5005F3ED0B3F5005F00F248
:10582C008780B3F5805F00F08580B3F5805F7FD80B
:10583C00702B1AD0702B7BD8602B50D0602B77D864
:10584C00502B3CD0502B73D8402B58D0402B6FD8BA
:10585C00302B64D0302B6BD8202B60D0202B67D80A
:10586C00002B5CD0102B5AD062E07B6818683B6828
:10587C0099683B685A683B68DB6800F0CAFA7B6839
:10588C001B689B68FB60FB6843F07703FB607B68DD
:10589C001B68FA689A604EE07B6818683B689968E8
:1058AC003B685A683B68DB6800F0B3FA7B681B689E
:1058BC009A687B681B6842F480429A603BE07B6884
:1058CC0018683B6859683B68DB681A4600F02AFA8E
:1058DC007B681B685021184600F081FA2BE07B682E
:1058EC0018683B6859683B68DB681A4600F048FA50
:1058FC007B681B686021184600F071FA1BE07B681E
:10590C0018683B6859683B68DB681A4600F00AFA6D
:10591C007B681B684021184600F061FA0BE07B683D
:10592C001A683B681B681946104600F058FA02E0EA
:10593C0000BF00E000BF7B68012283F83D207B683C
:10594C00002283F83C20002318461037BD4680BD4A
:10595C0080B485B000AF786039607B681B68FB60F1
:10596C007B68294A93420BD07B68B3F1804F07D0F8
:10597C007B68264A934203D07B68254A934208D120
:10598C00FB6823F07003FB603B685B68FA681343A9
:10599C00FB607B681C4A93420BD07B68B3F1804F51
:1059AC0007D07B68194A934203D07B68184A93420C
:1059BC0008D1FB6823F44073FB603B68DB68FA6832
:1059CC001343FB60FB6823F080023B685B69134365
:1059DC00FB607B68FA681A603B689A687B68DA62DD
:1059EC003B681A687B689A627B68074A934203D1CA
:1059FC003B681A697B681A637B6801225A6100BF95
:105A0C001437BD4680BC7047002C01400004004098
:105A1C000008004080B487B000AF786039607B68C4
:105A2C001B6A23F001027B681A627B681B6A7B612C
:105A3C007B685B683B617B689B69FB60FB6823F060
:105A4C007003FB60FB6823F00303FB603B681B687F
:105A5C00FA681343FB607B6923F002037B613B68AC
:105A6C009B687A6913437B617B681C4A93420CD117
:105A7C007B6923F008037B613B68DB687A6913431D
:105A8C007B617B6923F004037B617B68134A93423F
:105A9C0011D13B6923F480733B613B6923F40073A0
:105AAC003B613B685B693A6913433B613B689B69AB
:105ABC003A6913433B617B683A695A607B68FA68C0
:105ACC009A613B685A687B685A637B687A691A6288
:105ADC0000BF1C37BD4680BC704700BF002C014086
:105AEC0080B487B000AF786039607B681B6A23F0A4
:105AFC0010027B681A627B681B6A7B617B685B683F
:105B0C003B617B689B69FB60FB6823F4E043FB60B3
:105B1C00FB6823F44073FB603B681B681B02FA684C
:105B2C001343FB607B6923F020037B613B689B681C
:105B3C001B017A6913437B617B681D4A93420DD12B
:105B4C007B6923F080037B613B68DB681B017A690E
:105B5C0013437B617B6923F040037B617B68144AB0
:105B6C00934213D13B6923F480633B613B6923F47B
:105B7C0000633B613B685B699B003A6913433B6183
:105B8C003B689B699B003A6913433B617B683A69AC
:105B9C005A607B68FA689A613B685A687B689A63BA
:105BAC007B687A691A6200BF1C37BD4680BC70479F
:105BBC00002C014080B487B000AF786039607B68FE
:105BCC001B6A23F480727B681A627B681B6A7B6198
:105BDC007B685B683B617B68DB69FB60FB6823F07F
:105BEC007003FB60FB6823F00303FB603B681B68DE
:105BFC00FA681343FB607B6923F400737B613B6899
:105C0C009B681B027A6913437B617B681D4A934234
:105C1C000DD17B6923F400637B613B68DB681B025D
:105C2C007A6913437B617B6923F480637B617B68B6
:105C3C00144A934213D13B6923F480533B613B6973
:105C4C0023F400533B613B685B691B013A691343C6
:105C5C003B613B689B691B013A6913433B617B6861
:105C6C003A695A607B68FA68DA613B685A687B6803
:105C7C00DA637B687A691A6200BF1C37BD4680BC48
:105C8C00704700BF002C014080B487B000AF786033
:105C9C0039607B681B6A23F480527B681A627B68CC
:105CAC001B6A3B617B685B687B617B68DB69FB60C3
:105CBC00FB6823F4E043FB60FB6823F44073FB6058
:105CCC003B681B681B02FA681343FB603B6923F4B7
:105CDC0000533B613B689B681B033A6913433B6170
:105CEC007B680F4A934209D17B6923F480437B6123
:105CFC003B685B699B017A6913437B617B687A69BA
:105D0C005A607B68FA68DA613B685A687B681A6487
:105D1C007B683A691A6200BF1C37BD4680BC70476D
:105D2C00002C014080B487B000AFF860B9607A6095
:105D3C00FB681B6A7B61FB681B6A23F00102FB6832
:105D4C001A62FB689B693B613B6923F0F0033B6182
:105D5C007B681B013A6913433B617B6923F00A039F
:105D6C007B617A69BB6813437B61FB683A699A6112
:105D7C00FB687A691A6200BF1C37BD4680BC70474D
:105D8C0080B487B000AFF860B9607A60FB681B6ABA
:105D9C0023F01002FB681A62FB689B697B61FB684D
:105DAC001B6A3B617B6923F470437B617B681B033B
:105DBC007A6913437B613B6923F0A0033B61BB68A9
:105DCC001B013A6913433B61FB687A699A61FB6872
:105DDC003A691A6200BF1C37BD4680BC704780B45C
:105DEC0085B000AF786039607B689B68FB60FB68AE
:105DFC0023F07003FB603A68FB68134343F007031E
:105E0C00FB607B68FA689A6000BF1437BD4680BCA3
:105E1C00704780B487B000AFF860B9607A603B60BF
:105E2C00FB689B687B617B6923F47F437B613B68E8
:105E3C001A027B681A43BB6813437A6913437B616C
:105E4C00FB687A699A6000BF1C37BD4680BC7047FE
:105E5C0080B487B000AFF860B9607A60BB6803F0BB
:105E6C001F03012202FA03F37B61FB681A6A7B6948
:105E7C00DB431A40FB681A62FB681A6ABB6803F0C2
:105E8C001F03796801FA03F31A43FB681A6200BF17
:105E9C001C37BD4680BC704780B485B000AF7860BD
:105EAC0039607B6893F83C30012B01D1022346E02A
:105EBC007B68012283F83C207B68022283F83D201A
:105ECC007B681B685B68FB607B681B689B68BB60BE
:105EDC00FB6823F07003FB603B681B68FA68134394
:105EEC00FB607B681B68FA685A607B681B68164A03
:105EFC0093420ED07B681B68B3F1804F09D07B684E
:105F0C001B68124A934204D07B681B68104A934268
:105F1C000CD1BB6823F08003BB603B685B68BA683C
:105F2C001343BB607B681B68BA689A607B6801226C
:105F3C0083F83D207B68002283F83C200023184620
:105F4C001437BD4680BC7047002C01400004004053
:105F5C000008004080B582B000AF78607B68002BF1
:105F6C0001D101233FE07B6893F83D30DBB2002B7D
:105F7C0006D17B68002283F83C207868FCF7DCF9BA
:105F8C007B68242283F83D207B681B68DA687B6879
:105F9C001B6822F40052DA60786800F005F97B681F
:105FAC001B681A697B681B6822F490421A617B6833
:105FBC001B685A697B681B6822F02A025A617B684D
:105FCC001B68DA687B681B6842F40052DA607B68F5
:105FDC0000221A647B68202283F83D207B682022F3
:105FEC0083F83E20002318460837BD4680BD80B597
:105FFC008AB002AFF860B9603B601346FB800023A7
:10600C007B61FB6893F83D30DBB2202B7CD1BB6805
:10601C00002B02D0FB88002B01D1012375E0FB681B
:10602C0093F83C30012B01D102236EE0FB68012276
:10603C0083F83C20FB6800221A64FB68212283F859
:10604C003D20FCF7E7FA7861FB68FA889A84FB68D4
:10605C00FA88DA84FB689B68B3F5805F08D1FB682B
:10606C001B69002B04D10023FB61BB68BB6103E0FF
:10607C00BB68FB610023BB61FB68002283F83C20FA
:10608C002AE03B6800937B6900228021F86800F0CD
:10609C0040F80346002B01D0032336E0FB69002BAC
:1060AC000BD1BB691B881A46FB681B68C2F308023C
:1060BC005A60BB690233BB6107E0FB691A78FB6865
:1060CC001B685A60FB690133FB61FB68DB8C9BB27C
:1060DC00013B9AB2FB68DA84FB68DB8C9BB2002B29
:1060EC00CFD13B6800937B6900224021F86800F017
:1060FC0010F80346002B01D0032306E0FB68202296
:10610C0083F83D20002300E0022318462037BD46CB
:10611C0080BD80B584B000AFF860B9603B601346B9
:10612C00FB712CE0BB69B3F1FF3F28D0BB69002B9E
:10613C0007D0FCF76FFA02463B68D31ABA699A4249
:10614C001DD2FB681B68DA68FB681B6822F4D072EE
:10615C00DA60FB681B685A69FB681B6822F0010255
:10616C005A61FB68202283F83D20FB68202283F8CB
:10617C003E20FB68002283F83C2003230FE0FB68E1
:10618C001B681A68BB681340BA689A420CBF01239B
:10619C000023DBB21A46FB799A42C3D0002318467F
:1061AC001037BD4680BD000080B584B000AF78606C
:1061BC007B681B681B6923F440517B68DA687B6839
:1061CC001B680A431A617B689A687B681B691A43CF
:1061DC007B685B691343BB607B681B68DB6823F4DB
:1061EC00B05323F00C037A681268B9680B43D36080
:1061FC007B681B685B6923F440717B689A697B68D8
:10620C001B680A435A617B681B682C4A934203D172
:10621C00FDF790FEF86002E0FDF778FEF860FA6892
:10622C0013469B0013449A001A447B685B689B00DE
:10623C00B2FBF3F3224AA2FB03235B091901FA68B0
:10624C0013469B0013449A001A447B685B689B00BE
:10625C00B2FBF3F21A4BA3FB02035B09642000FBB5
:10626C0003F3D31A1B013233154AA2FB03235B0938
:10627C0003F0F0031944FA6813469B0013449A0088
:10628C001A447B685B689B00B2FBF3F20C4BA3FBDC
:10629C0002035B09642000FB03F3D31A1B013233A6
:1062AC00074AA2FB03235B0903F00F027B681B6800
:1062BC000A449A6000BF1037BD4680BD00380140CB
:1062CC001F85EB5180B582B000AF78600B467B80A8
:1062DC007A8841F2883379680348FEF757F800BF93
:1062EC000837BD4680BD00BF4C06002080B582B08B
:1062FC0000AF78600B467B807A8841F288337968EE
:10630C000348FEF77FF900BF0837BD4680BD00BFCC
:10631C004C06002080B500AF002210210948FDF783
:10632C00D8F9094B66221A70074B99225A70022130
:10633C000548FFF7C7FF012210210248FDF7C9F9F4
:10634C0000BF80BD00080140500A002080B500AF9E
:10635C00002210210848FDF7BCF9084B06221A70E0
:10636C0001210648FFF7AEFF012210210248FDF77C
:10637C00B0F900BF80BD00BF00080140500A0020EA
:10638C0080B500AF002210210848FDF7A2F9084B98
:10639C0004221A7001210648FFF794FF01221021F4
:1063AC000248FDF796F900BF80BD00BF0008014010
:1063BC00500A002080B483B000AF0346FB7100BFCD
:1063CC000C37BD4680BC704780B500AF0120FCF790
:1063DC002BF9002210211248FDF77BF9114B0522F5
:1063EC001A7001210F48FFF76DFF01210D48FFF7CF
:1063FC007DFF0C4B1A780C4B83F820200120FCF706
:10640C0013F9094B93F8203003F00103002BECD166
:10641C00012210210248FDF75CF900BF80BD00BFCE
:10642C0000080140500A00200C0A002080B500AF83
:10643C00FFF7CAFFFFF78AFF002210210B48FDF778
:10644C0048F90B4BC7221A7001210948FFF73AFF94
:10645C00012210210548FDF73CF9FFF7B5FFFFF7C6
:10646C008FFF0F20FFF7A6FF00BF80BD0008014083
:10647C00500A002080B584B000AFF860B9607A6033
:10648C003B60394B1B881A463B68934202D9364B0A
:10649C001B883B607A683B681344334A12889342EA
:1064AC0005D9314B1B881A467B68D31A3B602E4B9F
:1064BC001B881A46BB6802FB03F37A681344BB6063
:1064CC00FFF782FF0020FFF775FFFFF73FFF002269
:1064DC0010212648FDF7FDF8254B02221A70224B9D
:1064EC00DB7F002B17D0BB681B0EDAB2204B5A7027
:1064FC00BB681B0CDAB21E4B9A70BB681B0ADAB273
:10650C001B4BDA70BB68DAB2194B1A7105211848AB
:10651C00FFF7D8FE11E0BB681B0CDAB2144B5A70B3
:10652C00BB681B0ADAB2124B9A70BB68DAB2104B1A
:10653C00DA7004210E48FFF7C5FE3B689BB2194682
:10654C00F868FFF7BFFE012210210848FDF7C1F8DB
:10655C00FFF73AFFFFF714FF0F20FFF72BFF00BFE9
:10656C001037BD4680BD00BF0C0A0020000801405A
:10657C00500A002080B582B000AF104B9F221A70D9
:10658C00002210210E48FDF7A4F801210B48FFF75B
:10659C0099FE3B1D03211846FFF7A8FE012210218E
:1065AC000748FDF796F83B791A047B791B021343D5
:1065BC00BA79134318460837BD4680BD500A0020EF
:1065CC000008014080B584B000AF0346FB71FFF7B3
:1065DC00D1FFF8606420FCF727F8FFF79BFE6420DE
:1065EC00FCF722F8FB79002B16D04FF480530222D3
:1065FC0050495148FFF7FBFCFA685049504800F0ED
:10660C0043FA4F48F9F79CFD03469AB24FF4805376
:10661C004B494948FFF7EBFCFB689BB2FB60494BCD
:10662C000022DA77FB68A3F58043113B092B70D865
:10663C0001A252F823F000BF0F670008FF660008A4
:10664C00EF660008DF660008CF660008BF6600082A
:10665C00AF6600089D660008856600086D66000838
:10666C00384B0122DA77374B4FF480625A61364946
:10667C00334800F009FA7DE0324B0122DA77314BD6
:10668C004FF400725A6131492D4800F0FDF971E068
:10669C002C4B4FF480725A612D49294800F0F4F9C3
:1066AC0068E0284B80225A612A49254800F0ECF911
:1066BC0060E0244B40225A612749214800F0E4F95C
:1066CC0058E0204B20225A6124491D4800F0DCF987
:1066DC0050E01C4B10225A612149194800F0D4F9A2
:1066EC0048E0184B08225A611E49154800F0CCF9B5
:1066FC0040E0144B04225A611B49114800F0C4F9C4
:10670C0038E0104B02225A6118490D4800F0BCF9D0
:10671C0030E017490A4800F0B7F90948F9F710FDBD
:10672C0003469AB24FF4805305490348FFF75FFCC8
:10673C00D6E000BF487500088C0700204C75000897
:10674C00300A00200C0A00205875000870750008EB
:10675C0088750008A0750008B8750008D075000889
:10676C00E8750008007600081876000830760008F6
:10677C0048760008FB79002B0AD05B48F9F7E0FC5F
:10678C0003469AB24FF4805357495848FFF72FFCF1
:10679C00574B4FF480721A80554B4FF480529A60CD
:1067AC00534B5B691B01524AD360514BDB68504A17
:1067BC00926802FB03F34E4A1288B3FBF2F34C4A85
:1067CC0053604B4B9B681B01494A1361484BDB6878
:1067DC00474A926802FB03F39B0A454A9361FB7993
:1067EC00002B7DD0424B1B881A4642493E4800F094
:1067FC004BF93D48F9F7A4FC03469AB24FF4805389
:10680C0039493A48FFF7F3FB394B5B681A463A496A
:10681C00354800F039F93448F9F792FC03469AB23E
:10682C004FF4805330493148FFF7E1FB304B9B6804
:10683C001A4632492C4800F027F92B48F9F780FC0E
:10684C0003469AB24FF4805327492848FFF7CFFBF1
:10685C00274BDB681A462A49234800F015F92248D1
:10686C00F9F76EFC03469AB24FF480531E491F4849
:10687C00FFF7BDFB1E4B1B691A4622491A4800F054
:10688C0003F91948F9F75CFC03469AB24FF48053AC
:10689C0015491648FFF7ABFB154B5B691A461A49AD
:1068AC00114800F0F1F81048F9F74AFC03469AB287
:1068BC004FF480530C490D48FFF799FB0C4B9B6927
:1068CC001A461249084800F0DFF80748F9F738FC77
:1068DC0003469AB24FF4805303490448FFF787FBF1
:1068EC001037BD4680BD00BF300A00208C07002049
:1068FC000C0A00205C760008747600088876000884
:10690C00F4740008A0760008B8760008CC7600086D
:10691C0080B584B000AFF860B9607A603B60374BEB
:10692C001B881A463B68934202D9344B1B883B6048
:10693C007A683B681344314A1288934205D92F4B2D
:10694C001B881A467B68D31A3B602C4B1B881A4653
:10695C00BB6802FB03F37A681344BB60284B0B2221
:10696C001A70264BDB7F002B1FD0BB681B0EDAB2D4
:10697C00234B5A70BB681B0CDAB2214B9A70BB6864
:10698C001B0ADAB21E4BDA70BB68DAB21C4B1A71F6
:10699C001B4B00225A71002210211A48FCF799FE59
:1069AC0006211748FFF78EFC19E0BB681B0CDAB206
:1069BC00134B5A70BB681B0ADAB2114B9A70BB6846
:1069CC00DAB20F4BDA700E4B00221A710022102132
:1069DC000C48FCF77EFE05210948FFF773FC3B6869
:1069EC009BB21946F868FFF781FC0122102105487B
:1069FC00FCF76FFE00BF1037BD4680BD0C0A0020AF
:106A0C00500A002000080140014B1868704700BF75
:106A1C006400002070B500260C4D0D4C641BA410B6
:106A2C00A64209D100F09CFC00260A4D0A4C641BBE
:106A3C00A410A64205D170BD55F8043B9847013609
:106A4C00EEE755F8043B98470136F2E72C7B00083B
:106A5C002C7B00082C7B0008307B00080A449142F8
:106A6C0000F1FF3300D1704710B511F8014B914282
:106A7C0003F8014FF9D110BD03460244934200D1F3
:106A8C00704703F8011BF9E70EB46FF0004100B535
:106A9C009CB01DAB029006900791049108480949DF
:106AAC0053F8042B0591006802A9019300F068F8D3
:106ABC000022029B1A701CB05DF804EB03B0704707
:106ACC00640000200802FFFF2DE9F0478E68824623
:106ADC009E420C4690461F4638D88A8912F4906F15
:106AEC0032D0256809690133A5EB010965694B446E
:106AFC0005EB450505EBD5756D109D4238BF1D4660
:106B0C00530531D5294600F061FB064650B90C23DC
:106B1C004FF0FF30CAF80030A38943F04003A38143
:106B2C00BDE8F0874A462169FFF798FFA38923F453
:106B3C00906343F08003A38126614E4426603E4659
:106B4C006561A5EB0905A560BE4200D93E463246FB
:106B5C004146206800F0B8FAA36800209B1BA36094
:106B6C00236833442360DBE72A4600F0A3FB064688
:106B7C000028E1D15046216900F0C0FAC7E70000B7
:106B8C002DE9F04F98468B8907461B060D46144697
:106B9C009DB00ED50B6963B9402100F017FB28603E
:106BAC00286120B90C233B604FF0FF30D1E040232B
:106BBC006B610023099320238DF8293030234FF08B
:106BCC000109CDF80C80DFF8A4818DF82A3023461A
:106BDC009A4613F8012B0AB1252AF9D1BAEB040B0A
:106BEC000BD05B46224629463846FFF76DFF013035
:106BFC0000F0AA80099A5A4409929AF80030002BA6
:106C0C0000F0A28000234FF0FF32CDE905230AF1FA
:106C1C00010A049307938DF853301A9354460522B6
:106C2C0014F8011B514800F041FA049AD8B9D00667
:106C3C0044BF20238DF85330110744BF2B238DF80C
:106C4C0053309AF800302A2B15D0544600204FF0C0
:106C5C000A0C079A214611F8013B303B092B4ED9FF
:106C6C00B0B1079214E0A0EB080309FA03F3134345
:106C7C00A2460493D2E7039B191D1B680391002BBA
:106C8C00BBBF5B4242F0020207930793B8BF04926A
:106C9C0023782E2B0CD163782A2B35D1039B02340D
:106CAC001A1D1B680392002BB8BF4FF0FF330593DE
:106CBC00DFF8BCA003225046217800F0F7F940B170
:106CCC004023A0EB0A0003FA00F0049B01340343B9
:106CDC00049314F8011B062226488DF8281000F0A6
:106CEC00E5F9002838D0244B1BBB039B073323F05A
:106CFC00070308330393099B3344099367E70C4656
:106D0C0001200CFB0232A5E700234FF00A0C1946B8
:106D1C0001340593204610F8012B303A092A03D987
:106D2C00002BC5D00591C3E7044601230CFB0121C0
:106D3C00F0E703AB00932A463846104B04A9AFF397
:106D4C000080421C0646D6D1AB895B063FF52CAFC2
:106D5C0009981DB0BDE8F08F03AB00932A46384666
:106D6C00064B04A900F07CF8EBE700BFF87A0008AA
:106D7C00FE7A0008027B000800000000D56A0008BB
:106D8C002DE9F047164699468A680B6907469342E7
:106D9C00B8BF1346336091F843200C46DDF82080D1
:106DAC000AB1013333602368990642BF336802335A
:106DBC003360256815F0060506D104F1190AE3685D
:106DCC0032689B1AAB4228DC94F84320131E2268CD
:106DDC0018BF012392062DD44946384604F14302CC
:106DEC00C047013020D02368E56803F00603042B6C
:106DFC0018BF002532684FF00006A36808BFAD1A13
:106E0C00226908BF25EAE5759342C4BF9B1AED18A9
:106E1C001A34B5421AD1002008E0012352464946E3
:106E2C003846C047013003D14FF0FF30BDE8F08742
:106E3C000135C4E73020E11881F843005A1C94F85E
:106E4C0045102244023382F84310C5E70123224641
:106E5C0049463846C0470130E6D00136D9E7000034
:106E6C002DE9FF470F7E9146782F80460C469A46B7
:106E7C000C9D01F1430207D8622F0AD8002F00F0B5
:106E8C00D980582F00F0A48004F1420584F8427098
:106E9C003AE0A7F16303152BF6D801A151F823F0C2
:106EAC00056F0008196F0008956E0008956E0008B4
:106EBC00956E0008956E0008196F0008956E000815
:106ECC00956E0008956E0008956E000827700008F6
:106EDC00496F000809700008956E0008956E00084F
:106EEC0049700008956E0008496F0008956E0008FF
:106EFC00956E0008117000082B681A1D1B682A601B
:106F0C0004F1420584F842300123A4E0206829688A
:106F1C00060601F104030AD50E682B60002E03DA75
:106F2C002D23764284F843300A235E4819E00E681C
:106F3C0010F0400F2B6018BF36B2EFE72B682068BB
:106F4C00191D2960010601D51E6802E04606FBD515
:106F5C001E886F2F0CBF08230A235248002184F887
:106F6C0043106568002DA8BF2168A560A4BF21F05F
:106F7C00040121600EB9002D4DD01546B6FBF3F17E
:106F8C0003FB1167C75D05F8017D3746BB420E4612
:106F9C00F4D9082B0BD12368DE0708D52369616867
:106FAC009942DEBF302305F8013C05F1FF35521B39
:106FBC0022614B4621464046CDF800A003AAFFF7BC
:106FCC00DFFE01304CD14FF0FF3004B0BDE8F0874C
:106FDC00344881F845702968236851F8046B29609E
:106FEC001D0614D5DF0744BF43F0200323601EB9F0
:106FFC00236823F0200323601023AFE7236843F0BA
:10700C00200323607823284884F84530E3E75906A9
:10701C0048BFB6B2E6E71546BBE72B682668181DD5
:10702C006169286035061B6801D5196002E070069D
:10703C00FBD51980002315462361BAE72B68002184
:10704C001A1D2A601D686268284600F02FF808B1E6
:10705C00401B606063682361002384F84330A8E719
:10706C002A46494640462369D0470130ABD02368B5
:10707C009B0713D4E068039B9842B8BF1846A4E75B
:10708C000123324649464046D04701309BD001355A
:10709C00E36803995B1AAB42F2DCEBE7002504F1E1
:1070AC001906F5E7097B00081A7B0008034610B5A2
:1070BC00C9B202449342184601D1002003E004787F
:1070CC0001338C42F6D110BD884210B501EB02049D
:1070DC0002D98442234607D8431EA14208D011F896
:1070EC00012B03F8012FF8E7014602448A4200D134
:1070FC0010BD13F8014D02F8014DF7E738B5054600
:10710C00002940D051F8043C0C1F002BB8BFE418E8
:10711C0000F010F91C4A136833B9636014602846F8
:10712C00BDE8384000F00CB9A34208D920682118FA
:10713C008B4201BF19685B6809182160EDE71A469C
:10714C005B680BB1A342FAD911685018A0420BD15D
:10715C0020680144501883421160E0D118685B68C4
:10716C00014411605360DAE702D90C232B60D6E797
:10717C00206821188B4201BF19685B6809182160CF
:10718C0063605460CBE738BD5C0A002070B50E4ECE
:10719C000C463168054611B900F0BCF83060214648
:1071AC00284600F0B7F8431C0AD0C41C24F0030492
:1071BC00A04207D0211A284600F0ACF8013001D1CA
:1071CC004FF0FF34204670BD600A00202DE9F041DD
:1071DC00CD1C25F0030508350C2D38BF0C25002DD2
:1071EC00074601DBA94205D90C2300263B6030463B
:1071FC00BDE8F0812E4E00F09DF833681C4634BB80
:10720C0029463846FFF7C2FF431C04464DD134686B
:10721C002646002E40D123683146384604EB03083D
:10722C0000F078F880453AD1216803356D1A25F0C5
:10723C00030508350C2D38BF0C2538462946FFF7B9
:10724C00A5FF01302BD023682B4423600EE022686D
:10725C00521B1ED40B2A16D96119A342256018BFE4
:10726C005960636808BF316062514B60384604F165
:10727C000B0600F065F826F00706231DF21AB6D0AF
:10728C009B1BA350B3E76268A3420CBF32605A60E9
:10729C00ECE723466468B2E734467668B9E70C231A
:1072AC0038463B6000F04CF8A1E72560DEE700BFF4
:1072BC005C0A00202DE9F041804614460E4621B9A7
:1072CC001146BDE8F041FFF781BF2AB9FFF716FF61
:1072DC0025462846BDE8F08100F038F88442074680
:1072EC0002D8B4EB500F12D821464046FFF76EFF80
:1072FC0005460028EDD0BC422246314628BF3A460E
:10730C00FFF7ACFB31464046FFF7F8FEE1E73546A8
:10731C00DFE7000038B50023054D044608462B6016
:10732C00FBF7BEF8431C02D12B6803B1236038BDB8
:10733C00640A0020014800F011B800BF680A002060
:10734C00014800F00CB800BF680A002051F8043C5A
:10735C00181F002BBCBF0B58C018704770477047E4
:10736C00F8B500BFF8BC08BC9E467047F8B500BF26
:08737C00F8BC08BC9E467047F6
:1073840002030405060708090A0B0C0D0E0F101062
:1073940002030405060708090A0B0C0D0E0F101052
:1073A40049443A307825580A000000007732357194
:1073B400787820436869703A2077323571353132F4
:1073C4000A00000077323571787820436869703A92
:1073D40020773235713235360A0000007732357144
:1073E400787820436869703A2077323571313238C1
:1073F4000A00000077323571787820436869703A62
:10740400207732357136340A000000007732357146
:10741400787820436869703A207732357133320ABC
:107424000000000077323571787820436869703A3B
:10743400207732357131360A000000007732357119
:10744400787820436869703A207732357138300A89
:107454000000000077323571787820436869703A0B
:10746400207732357134300A0000000077323571EC
:10747400787820436869703A207732357132300A5F
:107484000000000077323571787820436869703ADB
:10749400207732357131300A0000000077323571BF
:1074A400787820556E6B6E6F776E2049440A000021
:1074B400506167652053697A653A202564204279D2
:1074C4007465730A000000005061676520436F759E
:1074D4006E743A2025750A00536563746F722053E5
:1074E400697A653A2025752042797465730A00002B
:1074F400536563746F7220436F756E743A202575FB
:107504000D0A0000426C6F636B2053697A653A2060
:1075140025752042797465730A000000426C6F631C
:107524006B20436F756E743A2025750A00000000C5
:1075340043617061636974793A202575204B420A6E
:10754400000000000D0A000049443A307825580D27
:107554000A00000077323571787820436869703A00
:1075640020773235713531320D0A000077323571AA
:10757400787820436869703A20773235713235362D
:107584000D0A000077323571787820436869703AC3
:1075940020773235713132380D0A00007732357177
:1075A400787820436869703A207732357136340D23
:1075B4000A00000077323571787820436869703AA0
:1075C400207732357133320D0A000000773235717D
:1075D400787820436869703A207732357131360DF6
:1075E4000A00000077323571787820436869703A70
:1075F400207732357138300D0A000000773235714A
:10760400787820436869703A207732357134300DC8
:107614000A00000077323571787820436869703A3F
:10762400207732357132300D0A000000773235711F
:10763400787820436869703A207732357131300D9B
:107644000A00000077323571787820556E6B6E6FC2
:10765400776E2049440D0A00506167652053697AAA
:10766400653A2025642042797465730D0A00000090
:107674005061676520436F756E743A2025750D0A55
:1076840000000000536563746F722053697A653A91
:107694002025752042797465730D0A00426C6F636E
:1076A4006B2053697A653A20257520427974657395
:1076B4000D0A0000426C6F636B20436F756E743A61
:1076C4002025750D0A0000004361706163697479B7
:1076D4003A202575204B420D0A00000000000000EE
:1076E400963007772C610EEEBA51099919C46D07CB
:1076F4008FF46A7035A563E9A395649E3288DB0E26
:10770400A4B8DC791EE9D5E088D9D2972B4CB60908
:10771400BD7CB17E072DB8E7911DBF906410B71DE5
:10772400F220B06A4871B9F3DE41BE847DD4DA1A1E
:10773400EBE4DD6D51B5D4F4C785D38356986C134F
:10774400C0A86B647AF962FDECC9658A4F5C0114C8
:10775400D96C0663633D0FFAF50D088DC8206E3BA6
:107764005E10694CE44160D5727167A2D1E4033CB8
:1077740047D4044BFD850DD26BB50AA5FAA8B535DF
:107784006C98B242D6C9BBDB40F9BCACE36CD832CE
:10779400755CDF45CF0DD6DC593DD1ABAC30D92675
:1077A4003A00DE518051D7C81661D0BFB5F4B42178
:1077B40023C4B3569995BACF0FA5BDB89EB8022875
:1077C4000888055FB2D90CC624E90BB1877C6F2FFA
:1077D400114C6858AB1D61C13D2D66B69041DC76F5
:1077E4000671DB01BC20D2982A10D5EF8985B171CE
:1077F4001FB5B606A5E4BF9F33D4B8E8A2C907787D
:1078040034F9000F8EA8099618980EE1BB0D6A7F13
:107814002D3D6D08976C6491015C63E6F4516B6BCC
:1078240062616C1CD83065854E0062F2ED95066C81
:107834007BA5011BC1F4088257C40FF5C6D9B065F6
:1078440050E9B712EAB8BE8B7C88B9FCDF1DDD6253
:10785400492DDA15F37CD38C654CD4FB5861B24DB9
:10786400CE51B53A7400BCA3E230BBD441A5DF4A83
:10787400D795D83D6DC4D1A4FBF4D6D36AE9694346
:10788400FCD96E34468867ADD0B860DA732D0444F1
:10789400E51D03335F4C0AAAC97C0DDD3C7105501C
:1078A400AA41022710100BBE86200CC925B56857C3
:1078B400B3856F2009D466B99FE461CE0EF9DE5E0C
:1078C40098C9D9292298D0B0B4A8D7C7173DB359BD
:1078D400810DB42E3B5CBDB7AD6CBAC02083B8ED4E
:1078E400B6B3BF9A0CE2B6039AD2B1743947D5EA5B
:1078F400AF77D29D1526DB048316DC73120B63E38A
:10790400843B64943E6A6D0DA85A6A7A0BCF0EE4E8
:107914009DFF099327AE000AB19E077D44930FF0A3
:10792400D2A3088768F2011EFEC206695D5762F79A
:10793400CB67658071366C19E7066B6E761BD4FED7
:10794400E02BD3895A7ADA10CC4ADD676FDFB9F9B4
:10795400F9EFBE8E43BEB717D58EB060E8A3D6D676
:107964007E93D1A1C4C2D83852F2DF4FF167BBD1A4
:107974006757BCA6DD06B53F4B36B248DA2B0DD8A7
:107984004C1B0AAFF64A0336607A0441C3EF60DF4A
:1079940055DF67A8EF8E6E3179BE69468CB361CB33
:1079A4001A8366BCA0D26F2536E2685295770CCC58
:1079B40003470BBBB91602222F260555BE3BBAC599
:1079C400280BBDB2925AB42B046AB35CA7FFD7C28A
:1079D40031CFD0B58B9ED92C1DAEDE5BB0C2649B7B
:1079E40026F263EC9CA36A750A936D02A906099CAE
:1079F4003F360EEB8567077213570005824ABF9521
:107A0400147AB8E2AE2BB17B381BB60C9B8ED292A3
:107A14000DBED5E5B7EFDC7C21DFDB0BD4D2D386FA
:107A240042E2D4F1F8B3DD686E83DA1FCD16BE816D
:107A34005B26B9F6E177B06F7747B718E65A08883E
:107A4400706A0FFFCA3B06665C0B0111FF9E658FCF
:107A540069AE62F8D3FF6B6145CF6C1678E20AA079
:107A6400EED20DD75483044EC2B30339612667A7FF
:107A7400F71660D04D476949DB776E3E4A6AD1AE4E
:107A8400DC5AD6D9660BDF40F03BD83753AEBCA9DD
:107A9400C59EBBDE7FCFB247E9FFB5301CF2BDBD4A
:107AA4008AC2BACA3093B353A6A3B4240536D0BA53
:107AB4009306D7CD2957DE54BF67D9232E7A66B3F0
:107AC400B84A61C4021B685D942B6F2A37BE0BB49D
:107AD400A18E0CC31BDF055A8DEF022D00000000A0
:107AE400000000000102030406070809000000006A
:107AF40001020304232D302B2000686C4C006566C2
:107B040067454647003031323334353637383941EA
:107B14004243444546003031323334353637383900
:087B2400616263646566000004
:047B2C00310100081B
:047B30000D0100083B
:107B34008B6C8740C3F55040FA7E224052B8FE3F1A
:107B44008716C93F3BDF9F3F0000803F5B424E3FAB
:107B54009031273F075F083F00000000FF0000004E
:107B64008B6C8740C3F55040FA7E224052B8FE3FEA
:107B74008716C93F3BDF9F3F0000803F5B424E3F7B
:107B84009031273F075F083F0024F40010000000F5
:107B94000100000068000020000000000000000058
:107BA40000000000000000000000000000000000D1
:107BB40000000000000000000000000000000000C1
:107BC40000000000000000000000000000000000B1
:107BD40000000000000000000000000000000000A1
:107BE4000000000000000000000000000000000091
:087BF400000000000000000089
:0400000508002525A5
:00000001FF
